:100000000C9455060C949C060C949C060C949C062F
:100010000C949C060C949C060C949C060C949C06D8
:100020000C949C060C949C060C940F310C94E331B8
:100030000C94D42A0C949C060C949C060C949C065C
:100040000C949C060C949C060C949C060C949C06A8
:100050000C949C060C942B2B0C949C060C949C06E4
:100060000C949C060C949C060C949C060C949C0688
:100070000C949C060C949C060C949C060C949C0678
:100080000C949C060C949C060C949C060C949C0668
:100090000C949C060C949C060C949C060C949C0658
:1000A0000C949C060C949C060C949C06726F775BD7
:1000B00025645D3A2025303458202D3E20253034EB
:1000C000580A006D61747269785F7363616E5F6373
:1000D0007573746F6D00657870616E6465727320FE
:1000E000696E697469616C697A65640A0069326372
:1000F0005F73746172742063616E6E6F74206164EB
:1001000064726573730A006932635F737461727439
:10011000204641494C45440A00636F6E666967207A
:1001200070696E73205355434345454445443A2016
:1001300025642C20616464723A20253032582C20CA
:10014000636D643A202530325820636F6E663A2022
:1001500025640A00636F6E6669672070696E73209C
:100160004641494C45443A2025642C206164647220
:100170003A20253032582C20636D643A20253032E5
:100180005820636F6E663A2025640A002900140027
:100190001A00080015001700000000002B4304009F
:1001A0001600070009000A0000000000E1001D0021
:1001B0001B0006001900050000000000E000E3003D
:1001C0004C0091642C410000000000001C0018004D
:1001D0000C00120013002D002A0000000B000D007F
:1001E0000E000F0033002800000000001100100076
:1001F0003600370052003800000000002C629042A8
:100200003800500051004F00000000003500140875
:100210001A08080815081708000000000100040863
:100220001608070809080A080000000001001D0858
:100230001B0806081908050800000000010001005D
:100240000100010001000000000000001C08180867
:100250000C08120813082E00010000000B080D08FE
:100260000E080F08340001000000000011081008FB
:100270002F0230024B00310000000000010001009D
:1002800031004A004E004D000000000001003A001D
:100290003B002000210022000000000001000100BE
:1002A0000100010001000100000000000100010048
:1002B0000100010001000100000000000100010038
:1002C00001000100010000000000000023002400E4
:1002D0002500260027002E0001000000010001007B
:1002E00001000100340001000000000001000100D5
:1002F0002F0030004B003100000000000100010021
:1003000031004A004E004D000000000001001E00B8
:100310001F003C003D003E00000000000100005CAA
:1003200001000100010001000000000001000100C7
:1003300001000100010001000000000001000100B7
:100340000100010001000000000000003F0040002B
:10035000410042004300440045000000010001004C
:1003600001000100C35CC25C00000000010001004C
:100370000100C95CC75CCA5C00000000010001000C
:100380000100C55CC85CC65C0000000044454255E5
:10039000473A2064697361626C65642E0A004445C3
:1003A0004255473A20656E61626C65642E0A000012
:1003B000000000000000002A2B28000000000000C0
:1003C0000000000000000000000029000000002CD8
:1003D0001E3420212224342627252E362D37382777
:1003E0001E1F202122232425263333362E37381F83
:1003F0000405060708090A0B0C0D0E0F1011121345
:100400001415161718191A1B1C1D2F3130232D35E2
:100410000405060708090A0B0C0D0E0F1011121324
:100420001415161718191A1B1C1D2F3130354C00C6
:1004300000000000000000000000000000000000BC
:1004400000000000000000000000000000000000AC
:100450000000007E0F00D4FFFFFFC7000000784FB0
:100460006E6573686F743A206163746976653A20CB
:1004700025640A000A0025303258006B6579626FE6
:100480006172645F7365745F6C65643A20000A0092
:100490002530313662003A200025303258000A7289
:1004A0002F632030313233343536373839414243C7
:1004B0004445460A00290A002575002F00257500CD
:1004C0005D280025640020002564002000256400CC
:1004D00020002564007C0025303258006D6F757354
:1004E000656B6579205B62746E7C7820792076205C
:1004F000685D287265702F61636C293A205B007219
:1005000067626C696768742074696D6572206469DC
:100510007361626C652E0A007267626C6967687449
:100520002074696D657220656E61626C65642E0A67
:10053000007267626C6967687420736574207370F9
:10054000656564205B4E4F454550524F4D5D3A20E6
:1005500025750A007267626C696768742073657438
:10056000207370656564205B454550524F4D5D3A80
:100570002025750A007267626C696768742073656C
:100580007420687376205B4E4F454550524F4D5D49
:100590003A2025752C25752C25750A007267626C2A
:1005A000696768742073657420687376205B4545BD
:1005B00050524F4D5D3A2025752C25752C25750A16
:1005C000007267626C69676874207261696E626F3D
:1005D0007720736574206873763A2025642C25642F
:1005E0002C25642C25750A007267626C6967687433
:1005F0002064697361626C65205B4E4F45455052C3
:100600004F4D5D3A207267626C696768745F636F13
:100610006E6669672E656E61626C65203D2025758A
:100620000A007267626C696768742064697361624A
:100630006C65205B454550524F4D5D3A20726762B4
:100640006C696768745F636F6E6669672E656E615B
:10065000626C65203D2025750A007267626C6967CF
:10066000687420656E61626C65205B4E4F45455035
:10067000524F4D5D3A207267626C696768745F63C0
:100680006F6E6669672E656E61626C65203D202520
:10069000750A007267626C6967687420656E6162D2
:1006A0006C65205B454550524F4D5D3A2072676244
:1006B0006C696768745F636F6E6669672E656E61EB
:1006C000626C65203D2025750A007267626C69675F
:1006D000687420746F67676C65205B454550524FA6
:1006E0004D5D3A207267626C696768745F636F6E14
:1006F0006669672E656E61626C65203D2025750A0E
:10070000007267626C69676874206D6F6465205B56
:100710004E4F454550524F4D5D3A2025750A0072A7
:1007200067626C69676874206D6F6465205B45451E
:1007300050524F4D5D3A2025750A007267626C6910
:100740006768745F696E6974207267626C69676854
:10075000745F636F6E6669672E6D6F6465203D2000
:10076000302E2057726974652064656661756C74FB
:100770002076616C75657320746F20454550524F2B
:100780004D2E0A007267626C696768745F696E69F2
:1007900074206565636F6E666967206973206E6F8C
:1007A0007420656E61626C65642E0A007267626C0B
:1007B000696768745F696E6974207374617274210B
:1007C0000A007267626C696768745F696E69742099
:1007D00063616C6C65642E0A007267626C6967689D
:1007E000745F636F6E6669672E7370656564203D24
:1007F0002025640A007267626C696768745F636FC2
:100800006E6669672E76616C203D2025640A007251
:1008100067626C696768745F636F6E6669672E7381
:100820006174203D2025640A007267626C69676804
:10083000745F636F6E6669672E687565203D20255D
:10084000640A007267686C696768745F636F6E66DC
:1008500069672E6D6F6465203D2025640A0072670C
:10086000626C696768745F636F6E6669672E656E38
:1008700061626C65203D2025640A007267626C69C4
:100880006768745F636F6E66696720454550524FB5
:100890004D3A0A007F3F1F643214643214783C1EC4
:1008A0001E140A052223252628292A2C2D2F303212
:1008B000333536383A3B3D3E4042434547494A4C42
:1008C0004E5051535557595A5C5E60626466686970
:1008D0006B6D6F71737577797B7D7F818385878978
:1008E0008A8C8E90929496989A9C9E9FA1A3A5A77D
:1008F000A8AAACAEAFB1B3B4B6B8B9BBBCBEBFC1A9
:10090000C2C3C5C6C7C9CACBCCCDCED0D1D2D2D333
:10091000D4D5D6D7D7D8D9D9DADADBDBDBDCDCDC47
:10092000DCDCDDDDDDDDDCDCDCDCDCDBDBDBDADA0A
:10093000D9D9D8D7D7D6D5D4D3D2D2D1D0CECDCC81
:10094000CBCAC9C7C6C5C3C2C1BFBEBCBBB9B8B696
:10095000B4B3B1AFAEACAAA8A7A5A3A19F9E9C9A21
:1009600098969492908E8C8A89878583817F7D7BEF
:1009700079777573716F6D6B6968666462605E5CD0
:100980005A5957555351504E4C4A49474543424096
:100990003E3D3B3A3836353332302F2D2C2A29282C
:1009A00026252322FFAA7F554000010101010101F4
:1009B0000101010202020202020202020303030316
:1009C00003030303040404040404040505050505E6
:1009D00006060606060707070707080808080909A4
:1009E00009090A0A0A0B0B0B0C0C0C0D0D0D0E0E4F
:1009F0000E0F0F0F101011111112121313141415E2
:100A00001516161717181819191A1A1B1B1C1D1D55
:100A10001E1E1F20202122222324242526262728AB
:100A200029292A2B2C2D2D2E2F30313232333435DB
:100A3000363738393A3B3C3D3E3F404142434445DE
:100A4000464748494A4C4D4E4F50515354555658BD
:100A5000595A5B5D5E5F616264656668696B6C6D67
:100A60006F7072737577787A7B7D7E8082838587DD
:100A7000888A8C8E8F91939596989A9C9EA0A2A31B
:100A8000A5A7A9ABADAFB1B3B5B7BABCBEC0C2C420
:100A9000C6C9CBCDCFD1D4D6D8DBDDDFE2E4E7E9E0
:100AA000EBEEF0F3F5F8FAFDFF0A0025303258209E
:100AB000006B6579626F6172645F7265706F7274EA
:100AC0003A20005B735D004B6579626F6172642050
:100AD00073746172742E0A005B575D005B535D0096
:100AE0005B525D005B445D005B435D001C034300A3
:100AF0006F006C0075006D006E00310033002D003A
:100B000061006E007300690000000E0341004200A6
:100B100070006C00750073000000040309040902F2
:100B20007B00040100A0FA09040000010301010098
:100B30000921110100012240000705810308000A74
:100B40000904010002030000000921110100012233
:100B5000220007058203200001070503032000018E
:100B60000904020001030000000921110100012213
:100B70007B000705840320000A0904030002030028
:100B80000000092111010001222200070585032030
:100B9000000107050503200001120100020000000A
:100BA0000801AB30C10100010200010631FF0974E8
:100BB000A1010975150026FF00952075088102091D
:100BC00076150026FF00952075089102C00660FF8B
:100BD0000961A1010962150026FF009520750881B1
:100BE000020963150026FF00952075089102C005D3
:100BF000010902A10185020901A1000509190129C4
:100C000008150025019508750181020501093009C3
:100C1000311581257F9502750881060938158125D2
:100C20007F950175088106050C0A38021581257F1C
:100C3000950175088106C0C005010980A1018503E1
:100C400019012AB700150126B7009501751081001A
:100C5000C0050C0901A101850419012AA002150192
:100C600026A002950175108100C005010906A101A9
:100C7000050719E029E7150025019508750181028E
:100C80009501750881010507190029FF150026FF48
:100C90000095067508810005081901290595057557
:100CA000019102950175039101C011241FBECFEF80
:100CB000DAE0DEBFCDBF04B603FE27C08091330368
:100CC00090913403A0913503B09136038730904B57
:100CD000A740B04BD1F4109233031092340310921A
:100CE00035031092360314BE84B7877F84BF0FB6D6
:100CF000F894A895809160008861809360001092BC
:100D000060000FBEE0E0F8E3099511E0A0E0B1E07B
:100D1000E2EEF8E602C005900D92A03DB107D9F7CA
:100D200023E0A0EDB1E001C01D92A333B207E1F7CB
:100D30000E9439190C9438340C940000FF93EF93FF
:100D4000E091D001F091D101309709F00995EF9130
:100D5000FF910895FC018591803011F0EFDFFBCF0A
:100D60000895FF27E0E230E247FF0CC0419597FF6E
:100D700009C0EDE26095709580959095611D711D9B
:100D8000811D911D27FF02C0219530E350E2AA2763
:100D9000660F771F881F991FAA1FA41710F0A41BA6
:100DA00063955A95A9F7AA3008F0A95FA05DAF93A3
:100DB000F395611571058105910541F7ED3211F447
:100DC000EF93F395F21718F43F93F395FBCF8F91C0
:100DD000B5DFFA95E1F70895E991F99185918030B1
:100DE00021F0853219F0AADFF9CF089520E0E894C8
:100DF00055915532C1F3503311F4689455915A33DB
:100E000048F4505390F3220F022E220F220F200D90
:100E1000250FF4CF0EF4219589919991533619F34A
:100E2000533729F1533559F1BC0188279927E894A4
:100E30005C3621F48991999168945591543639F42E
:100E400046EF7EF077FF0DC08FEF9FEF0AC055375A
:100E50004AE039F0583540E121F0523642E009F0DD
:100E60000895FF93EF937DDFEF91FF91B7CFFF934D
:100E7000EF93FC0181918030B9F360DFFBCFFF93EA
:100E8000EF9368DFF1CFDF93CF93CDB7DEB7259631
:100E9000A3DFCF91DF910895809144028160809318
:100EA000440264E080E091E00E94140980914402D1
:100EB00080FF04C086ED90E00C94AA0608957F920E
:100EC0008F929F92AF92BF92CF92DF92EF92FF925A
:100ED0000F931F93CF93DF93D82FC92F8091440294
:100EE00080FF04C083EC90E00E94AA060D2F1C2F07
:100EF00080E0C82E81E0D82ED0E0C0E0712C9CEAC2
:100F0000A92E90E0B92EF801E190F1908F01C60171
:100F10000E949D094C010097A9F0E816F90691F08E
:100F20009F928F93FF92EF92DF93CF93BF92AF92F6
:100F30000E944307EDB7FEB738960FB6F894FEBF90
:100F40000FBEEDBFF80132979182808281E0E814F4
:100F5000F90409F480E0782A2196F4E0CF0ED11C40
:100F6000C430D10581F6872DDF91CF911F910F916C
:100F7000FF90EF90DF90CF90BF90AF909F908F90B9
:100F80007F9008951092B90088E48093B800E4E659
:100F9000F0E080818F77808384E08093BC000895A7
:100FA000EF92FF920F931F93CF93DF93182FEB01D4
:100FB0001092BC0084EA8093BC000E94042B7C0148
:100FC0008091BC0087FF11C08091B900887F883074
:100FD00001F18091B900887F8031D9F0809144027D
:100FE00080FD12C08FEF9FEF08C0C7010E941C2B2D
:100FF0008C179D0728F38EEF9FEFDF91CF911F9104
:101000000F91FF90EF90089587E091E00E94AA066B
:10101000E9CF1093BB0084E88093BC000E94042BAE
:101020008C018091BC0087FF0EC08091B900887F41
:10103000883181F0803471F08091440280FFD2CFFA
:101040008DEE90E0E3CFC8010E941C2B8C179D070A
:1010500040F3D1CF90E080E0D0CF0F931F93CF9398
:10106000DF938B018093BB0084E88093BC000E94D7
:10107000042BEC018091BC0087FF11C02091B900C6
:10108000287F81E090E0283211F490E080E0919593
:1010900081959109DF91CF911F910F910895CE0114
:1010A0000E941C2B8017910728F38EEF9FEFF2CF41
:1010B0000F931F93CF93DF938C0184EC8093BC003C
:1010C0000E94042BEC018091BC0087FF08C0809136
:1010D000BB0090E0DF91CF911F910F910895CE0159
:1010E0000E941C2B8017910770F38EEF9FEFF2CFB9
:1010F0000F931F93CF93DF938C0184E88093BC0000
:101100000E94042BEC018091BC0087FF08C08091F5
:10111000BB0090E0DF91CF911F910F910895CE0118
:101120000E941C2B8017910770F38EEF9FEFF2CF78
:10113000CF92DF92EF92FF920F931F93CF93DF93A3
:10114000C62F6A017901B8010E94D00797FD0CC033
:10115000B8018C2F0E942D08E601EC0CFD1CCE1569
:10116000DF0511F097FF0CC024E92093BC00DF914C
:10117000CF911F910F91FF90EF90DF90CF90089546
:10118000B80189910E942D08EACFCF92DF92EF92A9
:10119000FF920F931F93CF93DF93F82EE62EEA0171
:1011A0006901B8010E94D00797FD15C0B8018E2DC6
:1011B0000E942D0897FD0FC0B8018F2D81600E94FD
:1011C000D007F12CE12C21E0C21AD108EC14FD0467
:1011D00000F597FF11C024E92093BC0018161906EA
:1011E00014F490E080E0DF91CF911F910F91FF9078
:1011F000EF90DF90CF900895C8010E94580897FDA6
:1012000004C0FE01EE0DFF1D80832FEFE21AF20AEB
:10121000DDCF97FDE0CFC8010E94780897FDDBCFB6
:10122000CC0DDD1D8883D7CF2F923F924F925F92D6
:101230006F927F928F929F92AF92BF92CF92DF92E6
:10124000EF92FF920F931F93CF93DF930F92CDB73F
:10125000DEB76C01362E8091D20181110EC081E083
:101260008093D2010E94C2072FEF89E698E12150B6
:1012700080409040E1F700C000007601B12C89E188
:10128000882E81E0982E94E5692E91E0792E222413
:101290002A94B31014C00F90DF91CF911F910F913A
:1012A000FF90EF90DF90CF90BF90AF909F908F9086
:1012B0007F906F905F904F903F902F900895F7012F
:1012C000A180D080DD0C5A2C550C5A0CC12CCA10B0
:1012D00005C0B394F4E0EF0EF11CDBCF452C4C0CB1
:1012E00029820AE010E021E030E0AE014F5F5F4F5D
:1012F000642D8D2D0E9498082981009799F01F92E6
:101300002F931F924F921F92DF929F938F937F9202
:101310006F920E9443070FB6F894DEBF0FBECDBF99
:10132000C394D5CF1F922F931F924F921F92DF929B
:101330001F921F929F928F92ECCFEF92FF920F938A
:101340001F93CF93DF9300D0CDB7DEB77C01FC01B4
:1013500080819FEF99839A83218130E00AE010E039
:10136000AE014F5F5F4F60E0880F0E94C508892B78
:1013700039F5F70121812150022E000C330B90E04A
:1013800080E027FF10C080959095F701228133817E
:10139000822393230F900F90DF91CF911F910F9194
:1013A000FF90EF900895E1E0F0E0EC0FFD1FE20FF9
:1013B000F31F4081642F782FCB0121503109E1CFF9
:1013C00090E080E0E7CF81E0089581E008950C94FB
:1013D000E50908950C94E9091F93CF93DF9300D09A
:1013E00000D00F92CDB7DEB749835A836B8330911B
:1013F000D30189819A8131111DC06623B9F022235E
:10140000A9F00E947E10182F682F89819A810E946E
:101410002B1069817A81812F0F900F900F900F9080
:101420000F90DF91CF911F910C94C0260E9457100E
:10143000182FEFCF0E947E1069817A81EDCFFC01D9
:10144000262F408151816281738184810C94EC0943
:1014500081E00895CF93DF93EC0160E00E941F0AC2
:10146000BE01DF91CF910C94EA09E1E0F0E0DF01E9
:1014700002C0AA0FBB1F6A95E2F7BD01DF0102C0DF
:10148000AA0FBB1F4A95E2F76A2B01C0EE0F2A95FF
:10149000EAF7962F9823961302C08E2B0895E095B5
:1014A0008E230895242F462F682F8091EC010E94EF
:1014B000350A0C94E80F0E945A180E94E60B0C940F
:1014C00075180C94781808950E94800F0E94630A82
:1014D0002FEF84E39CE0215080409040E1F700C072
:1014E00000000C944F2B0F931F93CF93DF938C012D
:1014F00061E00E941F0AEC01B8010E94A624882323
:1015000009F446C0B801CE010E94E709882309F416
:101510003FC0B801CE010E94F7278823C9F1B80166
:10152000CE010E944928882399F1B801CE010E947A
:101530006C29882369F1B801CE010E945D238823BC
:1015400039F1F8018281882361F0CE3DFCE5DF07A7
:10155000B9F170F4C115ECE5DE07C1F0C130DC452E
:10156000E9F0C801DF91CF911F910F910C94E3092D
:10157000CB358DE5D80751F1CC35EDE5DE0719F116
:10158000CA35DD4571F70E94EA13EBCF0E94640A69
:1015900080E0DF91CF911F910F91089590914402C7
:1015A000892F8E7F90FF81608093440280FF05C069
:1015B0008EE993E00E94AA06EBCF8CE893E0FACF85
:1015C0000E944A15E5CF0E94E113CBCF0E94ED1394
:1015D000C8CFDF92EF92FF920F931F93CF93DF93C9
:1015E000E82FF0E0E155FC4FD490282F2695269562
:1015F000269530E0F901E15BFB4F0491877010E024
:10160000082E02C0159507950A94E2F7017011277C
:10161000F901E15CFB4FE490F12C082E02C0F59437
:10162000E7940A94E2F791E0E922FF24F901E15DF1
:10163000FB4FC491D0E002C0D595C7958A95E2F7DB
:10164000C170DD270115110519F081EE0E94320CE1
:10165000E114F10419F086EE0E94320C8D2D0E94E7
:10166000310DEF2819F086EE0E94C40C012B19F001
:1016700081EE0E94C40CCD2B51F08CE2DF91CF9112
:101680001F910F91FF90EF90DF900C94310DDF913F
:10169000CF911F910F91FF90EF90DF900895EF92FF
:1016A000FF920F931F93CF93DF93EC01162F0AE065
:1016B0008881882309F454C0813009F04EC08981A3
:1016C000813099F47E0122E0E20EF11C8A810E94B1
:1016D000310DE7012196812F815050F3EFE9FFE0B2
:1016E0003197F1F700C00000F7CF823041F47E015E
:1016F00082E0E80EF11C8A810E94320CEACF83302E
:1017000041F47E01E2E0EE0EF11C8A810E94C40CDD
:10171000E0CF843011F02196DDCF2A81229690E02F
:1017200080E0AE014F5F5F4F2053330B2A3031050D
:1017300048F0019778F2EFE9FFE03197F1F700C048
:101740000000F7CF089FB001099F700D1124C90157
:10175000860F971F2981EA01E4CF0E94E90ABACFD8
:10176000DF91CF911F910F91FF90EF90089560E06E
:101770000C944F0B829590E09C01220F331F220F97
:10178000331F2C7C95958795959587958373282B8A
:1017900030E0C901880F991F8A7A359527952575FC
:1017A000822B0895CF93DF93D92F0E94BA0BC82FB5
:1017B0008D2F0E94BA0B9C2FDF91CF910895089531
:1017C0000C94DF0B81E008950C94E20B0895CF9305
:1017D000C82F0E94E00B8C2FCF910C94E40BCF9379
:1017E000DF93CDB7DEB72B970FB6F894DEBF0FBEF1
:1017F000CDBF4F83588769877A878B8761110E9495
:1018000010141E821D8285E0FE013796DE011196BE
:1018100001900D928A95E1F78C819D81892B89F445
:1018200049815A816B817C818D819E810E94FD124C
:101830002B960FB6F894DEBF0FBECDBFDF91CF91D0
:10184000089589819A8189238F3F51F3CE010196B2
:101850000E94280A8111E4CFEBCFFC0180819181A5
:101860000C94AB10CF93C82F882309F48BC0823817
:10187000C1F40E949B2981FD85C089E30E949713D2
:101880000E9433142FEF81EE94E02150804090406D
:10189000E1F700C0000089E30E949E13CF910C94F1
:1018A00033148338A1F40E949B2980FD6BC083E52B
:1018B0000E9497130E9433142FEF81EE94E0215081
:1018C00080409040E1F700C0000083E5E5CF843818
:1018D000A1F40E949B2982FD55C087E40E949713C2
:1018E0000E9433142FEF81EE94E02150804090400D
:1018F000E1F700C0000087E4CFCF8CEF8C0F813A76
:1019000090F46C2F80911001909111010E943F2A58
:10191000882329F08C2F0E949E130E9433148C2F51
:101920000E949713BBCF80E28C0F883048F4C770B9
:1019300081E001C0880FCA95EAF70E94F313AECF89
:10194000EBE5EC0FE33040F4F0E0EB59FE4F808123
:1019500090E0CF910C94012AE8E5EC0FE73150F4C8
:10196000F0E0EE0FFF1FE95CFE4F80819181CF9187
:101970000C94172AC03F30F08C2F0E94C719CF91CA
:101980000C949A1ACF910895882309F452C0823892
:1019900071F40E949B2981FF4CC089E30E94971338
:1019A0000E94331489E30E949E130C9433148338ED
:1019B00059F40E949B2980FF3CC083E50E94971345
:1019C0000E94331483E5EFCF843859F40E949B2999
:1019D00082FF2FC087E40E9497130E94331487E48C
:1019E000E2CF9CEF980F913AF0F290E2980F983086
:1019F00050F4877091E001C0990F8A95EAF7892F1A
:101A00000E94F913D2CF9BE5980F933020F490E019
:101A100080E00C94012A98E5980F973120F490E02B
:101A200080E00C94172A803F20F00E94211A0C9429
:101A30009A1A08951F93CF93DF93182FEB010E94FA
:101A4000320C209731F4812FDF91CF911F910C94AC
:101A5000C40C8FE99FE00197F1F700C000002197C7
:101A6000F0CF70E060E0893311F460E570E00C9431
:101A70001A0D882321F00E94F3130C943314089557
:101A8000882321F00E94F9130C9433140895BF9217
:101A9000CF92DF92EF92FF920F931F93CF93DF933A
:101AA0006C01D62FC72FFC011281058102950F70A2
:101AB0000E94B513E82E8823A1F0E12E112389F0AE
:101AC0008C2F807F803429F080E28D0FE12C8830CC
:101AD00040F082E00E9484140E94B51391E0E82E49
:101AE000E926BC2EB2949FE0B922FBE0FB1598F1E9
:101AF000EB2DF0E0E65CFB4C0C94D6330C2F0F7012
:101B0000C07F11F00295007F1123A9F0002359F046
:101B100080E28D0F883010F0D11109C0802F0E9413
:101B2000F3130E9433148D2F0E94320C14C0802FA7
:101B30000E940314F6CF8D2F0E94C40C002359F08D
:101B400080E28D0F883010F0D1112CC0802F0E94C0
:101B5000F9130E9433142B2D2850330B24303105F8
:101B600020F40E949B290E94E70BEE2009F469C132
:101B70000E94B11380FD65C1F60112820E94AB1371
:101B80000E94F90FC6010E94420F0E94AB13DF9121
:101B9000CF911F910F91FF90EF90DF90CF90BF906A
:101BA0000C940410802F0E940914D3CF2C2F2F7077
:101BB000F22EC07FC03219F0F29480EFF822DD23BC
:101BC00069F0D13049F1112391F1002351F1F6016F
:101BD000858180FFA8CF8F70858323C0112381F07A
:101BE000011106C00E9416148F290E94390DB3CF2F
:101BF0000130C1F70E9416148F290E941C14ABCF2C
:101C0000011106C00E9429148F2D0E94400DA3CF00
:101C1000013009F4A0CFF6CF112329F0063008F0E7
:101C20009ACF8F2DE2CF053008F095CFEDCF00236E
:101C300059F3D93349F4FFEF27EE33E0F150204058
:101C40003040E1F700C000008D2F0E94C40C83CF0C
:101C50008C2F86958695837069F0813009F07BCF53
:101C60008D2F9C2F9370111102C090E080E00E9494
:101C7000172A71CF8D2F9C2F9370111102C090E005
:101C800080E00E94012A67CF8D2F112329F00E9446
:101C9000C7190E949A1A5FCF0E94211AFACF8C2F7F
:101CA000837079F5111157CF4D2F429546954770A6
:101CB000440F440F8D2F8F70042E01C0880F0A949B
:101CC000EAF72D2F2071D4FF07C02FE030E001C0CC
:101CD000220F4A95EAF72095C695C695C370822BC8
:101CE000C23049F058F4C13019F00E94DA0F33CFF6
:101CF0000E94D50F30CF0E94DF0F2DCF0E94D30F4F
:101D00002ACF8695112311F08C2F8170882309F436
:101D100022CF4D2F429546954770440F440F8D2F8B
:101D20008F70042E01C0880F0A94EAF72D2F2071BE
:101D3000D4FF07C02FE030E001C0220F4A95EAF738
:101D40002095C695C695C370822BC23049F058F4D1
:101D5000C13019F00E942010FECE0E941B10FBCE55
:101D60000E942510F8CE0E94E80FF5CECF70112307
:101D700029F08C2F0E94F90F8D2F37CF8D2F0E94C5
:101D8000400D8C2F0E940410E6CED23F89F160F402
:101D9000D03FC9F0D13F29F1112309F442C001110C
:101DA000C2CE8C2F8F7121C0D33F39F1D43FA1F720
:101DB000112369F1CF718C2F0E94F90F63E08C2FF2
:101DC0000E946914C8CE112341F0053008F0C3CE3B
:101DD0008C2F8F710E941010BECE063008F0BBCE43
:101DE000F7CF8C2F8F71112369F20E94F90FB3CEB8
:101DF0008C2F8F711123C9F3C5CF112329F08C2F9C
:101E00008F710E94F10FA7CE0E94EE0FA4CE81E049
:101E10000E948414023008F49ECE82E00E94841452
:101E20009ACE002359F0D93309F00ECF8FEF97EEF9
:101E3000E3E081509040E040E1F704CF8C2F8F71B8
:101E4000A1CFDF91CF911F910F91FF90EF90DF9085
:101E5000CF90BF9008950F931F93CF93DF93EC0122
:101E6000688179818A810E94B5108C010E942A10B4
:101E70000E94D20FB801CE01DF91CF911F910F9137
:101E80000C94470DCF93DF93EC018B819C81892BC0
:101E900029F08881998189238F3F59F4DF91CF916F
:101EA0000895CE010E942B0FCE01DF91CF910C94AB
:101EB0002A0ACE010E94730A8111F3CF0E94B51342
:101EC000882361F38A81882349F382E0DF91CF91EF
:101ED0000C94841490E080E00E94012A90E080E05D
:101EE0000E94172A0E9410140E9413140E94331497
:101EF0000E94431C0C949A1A0E94A5130C946A0F1A
:101F00000E9400140C947C0FE92FE295EF70E250D0
:101F1000EE3070F4F0E0EA5BFB4C0C94D633803F7B
:101F200019F020F4883E20F481E00895843FE1F325
:101F300080E00895883EC0F3813FD1F7F5CF93FB51
:101F4000882780F90895FC01808191810E94AB105F
:101F50000C94840FCF93DF9300D000D00F92CDB7B5
:101F6000DEB70F900F900F900F900F90DF91CF91F1
:101F70000895CF93DF9300D000D000D0CDB7DEB767
:101F800026960FB6F894DEBF0FBECDBFDF91CF917E
:101F9000089508950C94C90F0E94CA0F8093ED0113
:101FA0000C946A0F08950C94CC0F9091ED01892B3D
:101FB0000C94CC0F9091ED0189230C94CC0F90914F
:101FC000ED0189270C94CC0F0C94C90F0C94E40FED
:101FD0000E94E60F8093EC010C946A0F80E00C9451
:101FE000E80F91E001C0990F8A95EAF7892F0C94C8
:101FF000E80F21E030E001C0220F8A95EAF78091D6
:10200000EC01822B0C94E80F21E030E001C0220F9C
:102010008A95EAF720958091EC0182230C94E80FD1
:1020200021E030E001C0220F8A95EAF78091EC01AF
:1020300082270C94E80F9091EC01892B0C94E80F07
:102040009091EC0189230C94E80F9091EC01892781
:102050000C94E80F08959295907F890F982F9770B0
:1020600041E001C0440F9A95EAF7869586958695DA
:1020700093E0899FF0011124EC52FE4F30E020E004
:1020800070E05191DF011197CB01022E02C09695AD
:1020900087950A94E2F781708195852784238527A7
:1020A0008C932F5F3F4F2330310559F70895929558
:1020B000907F890F982F977086958695869523E057
:1020C000829FF0011124EC52FE4F50E040E080E08E
:1020D000219130E0092E02C0369527950A94E2F747
:1020E00021703327042E01C0220F0A94EAF7822BB5
:1020F0004F5F5F4F4330510559F70895CF92DF92FC
:10210000FF920F931F93CF93DF936C010091EC012B
:102110008091ED01082BC7E0D0E010E0FC2EC80153
:102120000C2E02C0959587950A94E2F780FD0CC0AD
:102130002197A0F7F12C8F2DDF91CF911F910F9157
:10214000FF90DF90CF900895B6018C2F0E94641706
:10215000019771F3F0CFCF93DF93EC010E947E10D3
:10216000BE01DF91CF910C9464171F93CF93DF933F
:10217000EB019091D301992331F0CB01DF91CF9105
:102180001F910C94AB10882379F0CB010E947E1034
:10219000182F682FCE010E942B10BE01812FDF91D6
:1021A000CF911F910C946417CB010E945710182FE8
:1021B000F4CF1F93CF93DF93C091EE0116E080918F
:1021C000EF018C1304C0DF91CF911F910895D0E0EF
:1021D0001C9FF0011D9FF00D1124E051FE4F408126
:1021E000518162817381848195810E94B90F21960A
:1021F000C770E5CF409120025091210260912202E8
:102200007091230280912402909125020C94B90FC1
:102210001F93CF93DF9380912502807FA9F4809153
:102220002202882389F08091EE01C091EF01609134
:10223000200270912102A0912302B0912402D62F96
:10224000D72316E0C81304C0DF91CF911F910895E2
:1022500090E0109711F0DF3F19F401968770F2CFEC
:10226000189F9001199F300D1124F901E051FE4F84
:1022700041814713F2CF40814613EFCF4281411194
:10228000ECCF438154814A1B5B0B4A3F510528F731
:10229000809125028F70806180932502F901EB50B7
:1022A000FE4F80818F708061808380E292E00E9487
:1022B000420FDF91CF911F910C94D910AF92BF9232
:1022C000CF92DF92EF92FF920F931F93CF93DF9302
:1022D000CDB7DEB761970FB6F894DEBF0FBECDBFA6
:1022E0008C0185E0F801DE011D9601900D928A9522
:1022F000E1F7F801E28080E2C82E82E0D82E6091FA
:102300002302709124026115710509F45AC190915C
:10231000200220912102892F82238F3F09F451C18D
:1023200040815181A380B480F0902202F501E61B28
:10233000F70BFF2009F4F6C080912502382F307F7B
:10234000EA3FF10508F0AFC0311179C0FE2C25132A
:1023500023C0941321C0E1101FC08F70806180934F
:1023600025020E94FA10C6010E94420F80912502A8
:10237000F80185838F2D61960FB6F894DEBF0FBEEE
:10238000CDBFDF91CF911F910F91FF90EF90DF9024
:10239000CF90BF90AF900895AB2829F0842F85236C
:1023A0008F3F09F027C180E0F82FF170DF2E80FF0A
:1023B0003CC08091EE012091EF0136E0821315C000
:1023C0004D875E878D859E850E94AB10292F2295B3
:1023D0002F702230F0F0243018F59F70F1F0F801E2
:1023E0009581907FD1F4D12C1EC090E0389FF001F0
:1023F000399FF00D1124E051FE4F6181651306C035
:102400006081641303C06281E6120FC00196877079
:10241000D5CF9F7011F0882331F3805E883018F398
:10242000C8010E94420FFD2CA5CFEE2009F4A2CFD7
:1024300080912502816080932502F12C9BCF25138A
:1024400006C0941304C0F801EE2009F487C0C80147
:102450000E94A30F882319F1EE2009F18091250233
:10246000803270F0209120023091210238872F8332
:102470001986BB86AA868C87CE0107960E94420FDA
:1024800086E0F801A0E2B2E001900D928A95E1F7B2
:102490000E9408110E94FA10FF24F3946BCFC80128
:1024A0000E94420FF9CF311113C07A2DB98AA88A40
:1024B0006E2D89890E94AA0F80E292E00E94420F4D
:1024C00086E0F60111928A95E9F70E94FA10B5CFDD
:1024D00025130FC094130DC0E1100BC0F8018583C4
:1024E000C8010E94420F86E0F60111928A95E9F731
:1024F00041CFC8010E94A30F882389F2EE2079F210
:1025000080912502803208F4BBCF209120023091C7
:1025100021023A8329831B82BD82AC828E83CE0145
:102520000196ACCFEA3FF10508F03EC0FE2CEE204C
:1025300009F4B5CF25132AC0941328C08091250231
:1025400080FD1BC0982F907FC1F0F8018583903FDC
:1025500031F0982F907F905F8F70892B8583C80111
:102560000E94420F86E0F801A0E2B2E001900D92D5
:102570008A95E1F70E94FA10FDCE86E0F801A0E20C
:10258000B2E001900D928A95E1F7F4CEC8010E9465
:10259000A30F811175CF8091250281608093250260
:1025A000C8010E94420FE6CE7A2DB98AA88A6E2D04
:1025B00089890E94AA0F86E0F60111928A95E9F7AF
:1025C000D9CFEE2009F46BCFC8010E94A30FF82EDB
:1025D000882309F464CF86E0F801A0E2B2E001901C
:1025E0000D928A95E1F780E292E00E942D0C0E9404
:1025F0000811C0CF81E08E25D7CE1F93CF93DF93F4
:10260000CDB7DEB72C970FB6F894DEBF0FBECDBFA7
:102610004F83588769877A878B879C87CE01079677
:102620000E945E11882369F08A859B85892B39F089
:102630004F815885842F85238F3F09F071C016E0A4
:102640005FC086E0FE013796DE01119601900D9283
:102650008A95E1F78A859B85892B89F38F819885F7
:1026600089238F3F61F32091EF0130E0C90101968A
:10267000877099274091EE014817190671F40E945E
:10268000800F1092EF011092EE0186E0E0E2F2E09E
:10269000DF011D928A95E9F7D2CF96E0929FD00193
:1026A000939FB00D1124A051BE4FFE0131960190B1
:1026B0000D929A95E1F78093EF010E94D910BFCF58
:1026C000819FC001112480519E4F0E945E1188237A
:1026D000E9F0E091EE011E9FF0011124E051FE4F60
:1026E0004081518162817381848195810E94B90FFB
:1026F0008091EE0190E00196877099278093EE011A
:102700008091EE019091EF018913DACF2C960FB6EC
:10271000F894DEBF0FBECDBFDF91CF911F9108951A
:1027200069857A858B859C850E94B90F88CF682F33
:1027300080911001909111010C94752A682F80915D
:102740001001909111010C94772A809110019091C1
:1027500011010C94792A809126028595859585959D
:1027600008958091260287700895909126029770AF
:1027700081E009F480E00895CF93C82F80917C0216
:1027800082FB992790F99C17D1F0C0FB82F98093C6
:102790007C0280917B0290917C020E94C714809100
:1027A000440280FF0CC01F92CF938FE594E09F936B
:1027B0008F930E9443070F900F900F900F90CF912F
:1027C000089580917C0282FB882780F991E0892717
:1027D0000C94BC1381E00C94BC1380E00C94BC13EB
:1027E00080913202089590913202892B80933202B7
:1027F0000895809590913202982390933202089523
:1028000010923202089590913102892B8093310207
:102810000895809590913102982390933102089504
:10282000109231020895109230020895809127028B
:10283000089508950C94191490917C0292FD08C09B
:1028400090912702981721F0809327020C941A1474
:10285000089580912702882329F01092270280E0B2
:102860000C941A140895E0911001F09111018091D7
:1028700032028083E0911001F091110180819091EA
:102880003102892B8083E0911001F0911101808148
:1028900090913002892B808390912702992381F0B7
:1028A000E0911001F09111018081892B808380914A
:1028B0001001909111010E942D2A81110E9429146A
:1028C00080911001909111010C94A72908950C9406
:1028D000661490917C0292FD10C098E0899F90014F
:1028E0001124622B609326020E94F90F8091260228
:1028F0008595859585950C9467140C94F90F109225
:10290000260280E00C94671490912602809589231A
:1029100080932602282F277039F4282F082E000CC8
:10292000330B9217130621F490917C0292FF07C09B
:102930008595859585950E9404100C947F140895C3
:102940006FEF7FEF90E080E00C94223490E080E025
:102950000E94FE33893E9E4F11F40C944F2480E078
:10296000089582E090E00C94F03383E090E00C94C2
:10297000F033CF9384E090E00E94F033C82F82E2DE
:1029800090E00E94F033982F8C2FCF910895CF9331
:10299000C92F682F84E090E00E9404346C2F82E2FB
:1029A00090E0CF910C940434AB01BC018FE090E037
:1029B0000C941634AB01BC0183E190E00C94163406
:1029C00060E070E0CB010C94DA1460E070E0CB01C1
:1029D0000E94D4140C94E01469EE7EEF90E080E045
:1029E0000E94223460E082E090E00E94043460E0C3
:1029F00083E090E00E9404341092ED0160E084E0F6
:102A000090E00E94043460E082E290E00E9404348E
:102A100060E085E090E00E94043460E086E090E0B1
:102A20000E9404346FEF87E090E00E94043440E09D
:102A300050E0BA0188E090E00E94163460E08DE03A
:102A400090E00E94043440E050E0BA0188E190E058
:102A50000E94163460E087E190E00E94043440E078
:102A600050E0BA018CE190E00E94163470E060E022
:102A700080E290E00E94223440E050E0BA0188E118
:102A800090E00E94163480E00E9468240E948E2408
:102A90000C94E5140C94EC14682F8EE090E00C94E8
:102AA00004340E94102B6093400270934102809383
:102AB00042029093430260933C0270933D028093E4
:102AC0003E0290933F02089585B7806885BF85B721
:102AD000806885BF0895089508950C946B15089536
:102AE0000C946F150E9464158DE59DE20E94732B76
:102AF0000E946C150C946D1581E008950C947C1562
:102B0000089508950E9480150C9481150E94FB2A57
:102B10000E949D240E94CA180E94DA210C9470150C
:102B2000CF93C82F8091440282FF1EC080FF1CC03B
:102B30008BE794E00E94AA068091440280FF14C0B3
:102B40001F92CF9386E794E09F938F930E94430751
:102B5000809144020F900F900F900F9080FF04C05F
:102B600084E794E00E94AA068C2FCF910C94E70B87
:102B70008F929F92AF92BF92CF92DF92EF92FF928D
:102B80000F931F93CF93DF93CDB7DEB72A970FB67E
:102B9000F894DEBF0FBECDBF0E94EC1881110E94D9
:102BA000511554E3852E52E0952E10E000E0A02E42
:102BB000802F0E947A186C01F401E190F1904F018E
:102BC000E816F90609F45EC08091440281FD0E9476
:102BD0008318C7018C259D25B12CEE24E394F12C9C
:102BE0009C012E213F21232B09F446C00E947E1513
:102BF0008823A9F0BE82AF82CE20DF2081E0CD28DD
:102C000009F480E088870E94042B8160782F9A87DE
:102C100089874E815F8168858A850E94EF0B000F4E
:102C2000111FF801EC5CFD4F80819181E826F926A7
:102C3000F182E0820E94C6220E94371B0E949B29DB
:102C4000909133028917A9F10E949B298093330246
:102C50002A960FB6F894DEBF0FBECDBFDF91CF919D
:102C60001F910F91FF90EF90DF90CF90BF90AF90AA
:102C70009F908F900C949015B394EE0CFF1CF0E194
:102C8000BF12AECF0F5F1F4F0430110509F08FCF79
:102C90008FEF89838A831B820E94042B8160782FA7
:102CA0009D838C8349815A816B818D810E94EF0BBA
:102CB000C1CF2A960FB6F894DEBF0FBECDBFDF910D
:102CC000CF911F910F91FF90EF90DF90CF90BF9029
:102CD000AF909F908F900895CF93DF930E946817D5
:102CE000EC01811521E5920708F042C0811530E51D
:102CF000930708F09DC0883E910530F5803E910510
:102D000008F092C0883A910588F4853A910508F058
:102D100084C08130910509F487C0009709F484C00C
:102D2000049708F081C0D0E0C0E07EC08F3B9105E1
:102D3000D0F7C85AD0E0CC0FDD1FC859DE4F09903C
:102D4000D881C02DD46470C08115904250F4C11553
:102D500081E0D80708F068C0C03FD10520F3D065F6
:102D600063C0C11590E4D907F0F2DF70D06A5CC08F
:102D7000811525E5920700F5811534E5930708F0E4
:102D80008BC0811543E5940708F073C0C11582E537
:102D9000D80708F469C0CE018370992721E030E09C
:102DA00002C0220F331F8A95E2F7C695C69580E2CE
:102DB000C89FE001112454C0C11599E5D907A8F4B2
:102DC000C11528E5D20708F06CC0C11536E5D30758
:102DD00008F0A9CF8C2F0E94FF17C82FD0E0DC2F5E
:102DE000CC27CC27DF71D0621FC0C1154AE5D407BC
:102DF00008F45CC0CE0190568115904208F093CF44
:102E00008D2F8F710E94FF1790E0982F88278827B9
:102E10009F719C012C2BE901E6CFC55AD0E0CA5620
:102E2000DE4FC881D0E0D064CE01DF91CF9108950C
:102E3000E4E096958795EA95E1F783702C2F269527
:102E40002695237040E2249F90011124382B8C2F6B
:102E50008370C1E0D0E002C0CC0FDD1F8A95E2F79D
:102E6000C22BD32BDC68E0CFDC2FCC27C16FD06A1C
:102E7000DBCF8370992721E030E002C0220F331F9F
:102E80008A95E2F7C695C69590E2C99FE0011124A4
:102E9000C22BD32BDA68C8CFD82FCC27C46FD06A07
:102EA000C3CFDC2FCC27C06FD06ABECF8C2F8F70E2
:102EB0000E94FF1734E0D695C7953A95E1F7CF7099
:102EC0009C2FEC01D069B0CF0E94C0260C946C16E8
:102ED00082389105B1F1B0F48133910509F475C0E0
:102EE00048F48932910509F469C08A32910509F4E0
:102EF00073C008958533910509F459C0893391054C
:102F000001F10895833E9105A9F138F4803E9105C1
:102F1000F9F0823E910549F10895863E9105A9F1A7
:102F2000873E9105C9F1843E910519F520917C02F7
:102F300021FF1FC080917B0284FD14C087EE90E0CA
:102F4000089520917B022370A1F080EE90E0089517
:102F500020917B0220FD47C030917C0230FF09C0E8
:102F600024FF44C090E080E004C020917B0222FD59
:102F7000F7CF089520917B0222FD3BC030917C0267
:102F800030FDE3CF24FFF5CFEDCF20917B0223FF6F
:102F9000F0CF24FDE7CFD2CF20917B0223FD2CC0C0
:102FA00030917C0231FFEECF84EE90E008952091C5
:102FB0007B0225FFDECF89E290E0089520917B021D
:102FC00025FFD7CF85E390E0089520917B0226FF6F
:102FD000D0CF8AE290E0089520917B0226FFC9CFEE
:102FE00081E390E0089589E390E0089583EE90E016
:102FF000089582EE90E0089586EE90E00895909115
:103000007B0292FF06C0282F28712830F9F4877FB1
:10301000846093FF06C0282F28712831F1F4877E41
:10302000846120917C0220FF06C0382F387138302F
:10303000D9F4877F816021FF06C0282F28712831AD
:10304000D1F4877E816194FD877E0895282F2471B5
:103050002430F9F68B7F8860DCCF282F247124314F
:1030600001F78B7E8861DDCF382F3171313019F750
:103070008E7F8860E0CF282F2171213121F78E7E4D
:103080008861E1CF0C94A0140E94EC188FE39CE9B6
:103090000197F1F700C000000E94EC1880E00E9448
:1030A0007A1880FF04C00E9442180C944F2B089598
:1030B0000C9444180E94A614811102C00E944A1563
:1030C0000E94B114809344020E94B91490937C0230
:1030D00080937B020E9458180E94B5140E94D30F5F
:1030E0008091EC010C94E60F08950C9474180895E7
:1030F0000C947718E82FF0E0EE0FFF1FEB57FD4F11
:10310000808191810895CF92DF92EF92FF920F9389
:103110001F93CF93DF938EE994E00E94AA0685E87F
:10312000E82E82E0F82ED0E0C0E099E9C92E94E0C4
:10313000D92E00E914E0DF93CF93DF92CF920E9463
:10314000430786E994E00E94AA06F70181919191D4
:103150007F010E94D20B9F938F931F930F930E9426
:1031600043078EE894E00E94AA0621968DB79EB789
:1031700008960FB6F8949EBF0FBE8DBFC430D10520
:10318000D1F6DF91CF911F910F91FF90EF90DF90DB
:10319000CF9008950E944C07ADE7B2E011961C92C3
:1031A0001E92E5E8F2E01182108213961C921E92A4
:1031B00012971382128215961C921E9214971582F2
:1031C000148217961C921E9216971782168284E01C
:1031D0000E94FF180C945B0ACF938DE792E00E9447
:1031E0005F07C82F282F44E065E872E08DE792E082
:1031F0000E9400190E94610A8C2FCF9108950895B2
:10320000FF920F931F93CF93DF93F82E092F162F62
:10321000D72FC42F222349F081E0809347020E94D8
:10322000042B9093460280934502809147028823A5
:10323000A1F080914502909146020E941C2B0597B7
:1032400060F0EF2DF02FA12FBD2F90E080E0D0E0B7
:103250008C179D0744F010924702DF91CF911F9188
:103260000F91FF900895219131912D933D930196F7
:10327000EFCF0E94802A0E94BF2D0E94D82D0E946D
:10328000EE2D0E948215FBCF80914E0280FF12C06E
:103290006091170185E0689FB001112475956795CD
:1032A0007595679560387105A8F561157105A1F1EF
:1032B000862F089581FF09C06091170185E0689FFE
:1032C000B001112475956795EDCF6091170182FDCE
:1032D0000AC080914D028823D1F09091160160912F
:1032E0001701891728F085E0689FB0011124DACF13
:1032F000869FB001112485E0869F9001879F300D45
:103300001124692F70E0C9010E94C233CBCF65E060
:1033100070E0CECF8FE7089581E0089580914E024E
:1033200080FF0CC06091130170E0759567957595ED
:1033300067956115710549F1862F089581FF06C0D3
:103340006091130170E075956795F3CF609113015B
:1033500082FD0BC090914C029923A1F06091120163
:1033600080911301961738F0682F70E0603871056E
:1033700000F38FE70895899FC001112470E00E9437
:10338000C233F4CF61E070E0D7CF81E00895803F91
:1033900031F40E9444198195809352020895813F2F
:1033A00019F40E944419F8CF823F31F40E94441965
:1033B0008195809351020895833F19F40E94441926
:1033C000F8CF893F29F40E948E1980935302089503
:1033D0008A3F21F40E948E198195F7CF8B3F31F4FB
:1033E0000E948E1981958093540208958C3F19F4A0
:1033F0000E948E19F8CF9CE0980F953070F4845F8E
:10340000990B21E030E001C0220F8A95EAF7809104
:103410005002822B8093500208958D3F31F48091A9
:103420004E02816080934E0208958E3F21F4809178
:103430004E028260F7CF8F3FB9F780914E028460D1
:10344000F1CF40915102803F59F48091520287FFA1
:103450000DC01092520241110BC010924D0208C0D3
:10346000813F81F48091520218169CF3442381F02D
:103470008091530290915402892B09F05AC0109206
:103480004C020895823F49F447FFF0CF1092510259
:10349000809152028111ECCFE0CF833F19F41416D2
:1034A000ACF3E4CF90915302893F29F41916F4F656
:1034B00010925302DBCF8A3F19F497FFD7CFF8CF92
:1034C000909154028B3F29F497FFD0CF1092540271
:1034D000CDCF8C3F19F41916CCF3C8CF9CE0980FD0
:1034E000953090F4845F990B21E030E0B90102C07F
:1034F000660F771F8A95E2F7CB0180959091500275
:10350000892380935002B2CF8D3F31F480914E02D7
:103510008E7F80934E02AACF8E3F21F480914E027F
:103520008D7FF7CF8F3F09F0A1CF80914E028B7F27
:10353000F0CF08958091440283FF7EC08CED94E02B
:103540000E94AA06809150021F928F9387ED94E00B
:103550009F938F930E94430785ED94E00E94AA06F3
:1035600080915102282F082E000C330B3F938F932C
:1035700082ED94E09F938F930E94430780ED94E047
:103580000E94AA0680915202282F082E000C330BAD
:103590003F938F938DEC94E09F938F930E9443070A
:1035A0008BEC94E00E94AA0680915302282F082EEB
:1035B000000C330B3F938F9388EC94E09F938F9391
:1035C0000E94430786EC94E00E94AA068091540270
:1035D000282F082E000C330B3F938F9383EC94E03D
:1035E0009F938F930E94430780EC94E00E94AA0669
:1035F00080914D021F928F938DEB94E09F938F9358
:103600000E9443078BEB94E00E94AA0680914E0231
:103610001F928F9388EB94E09F938F930E944307B0
:1036200085EB94E00E94AA068DB79EB74C960FB624
:10363000F8949EBF0FBE8DBF0E94042B9C019091F9
:10364000510280915202982B21F030934B0220932B
:103650004A029091530280915402982B21F03093AA
:103660004902209348028FE492E00C94F329EF92F0
:10367000FF920F931F93CF93DF9300D000D000D021
:10368000CDB7DEB786E0EFE4F2E0DE0111960190FF
:103690000D928A95E1F7E0905102F090520200916C
:1036A0005302109154021092510210925202109241
:1036B0005302109254028E2D8F2991F080914A026C
:1036C00090914B020E941C2BAC0190914D029923CA
:1036D00009F43FC0809118018417150608F447C00B
:1036E000802F812B91F080914802909149020E9495
:1036F0001C2BAC0190914C02992309F477C0809166
:1037000014018417150608F47FC08091510290912E
:103710005202892B90915302892B90915402892B4C
:1037200011F00E949A1A86E0FE013196AFE4B2E0F1
:1037300001900D928A95E1F726960FB6F894DEBFB8
:103740000FBECDBFDF91CF911F910F91FF90EF90F2
:103750000895209119018AE0289F900111242417CF
:10376000350708F0BDCF9F5F90934D0202C09F3F89
:10377000D1F7EE2059F00E9444199FEF1E140CF46B
:1037800091E0899F802D112480935102FF2059F0F0
:103790000E9444199FEF1F140CF491E0899F802D23
:1037A00011248093520230915102332309F498CFAF
:1037B00020915202222309F493CF45EB3403C00138
:1037C0001124992359F09093510245EB2403900161
:1037D0001124332339F03093520282CF81E0809359
:1037E0005102F3CF81E0809352027ACF20911501EC
:1037F0008AE0289F900111242417350708F085CF0F
:103800009F5F90934C0202C09F3FD1F7002359F075
:103810000E948E199FEF10160CF491E0899F802D65
:10382000112480935302112359F00E948E199FEFA7
:1038300011160CF491E0899F802D1124809354027D
:1038400030915302332309F460CF20915402222394
:1038500009F45BCF45EB3403C0011124992359F0DF
:103860009093530245EB240390011124332339F044
:10387000309354024ACF81E080935302F3CF81E02A
:103880008093540242CF86E0EFE4F2E0DF011D9224
:103890008A95E9F710924D0210924C0210924E0256
:1038A0000895EF92FF920F931F93CF93DF93EB0155
:1038B000E82FD11110C0442321F0F0E0E755F64F76
:1038C000E4916E2F7E2F8E2FDF91CF911F910F915C
:1038D000FF90EF9008950D2F10E0282F30E0442343
:1038E00029F02755364FF901249130E0F6E0CF9FBB
:1038F000C0011124EFEFF0E0BF010E94AE33AB0135
:103900008C2F90E0880F991FA5E5A49FB001A59F7B
:10391000700D1124861B970B982F990F980FBF01DC
:10392000601B710B629FD001639FB00D729FB00D41
:1039300011248B2F9D9FB0011124672F7727EF0152
:10394000C61BD70BBE01629FE001639FD00D729F23
:10395000D00D11247F01E91AF108E09EB001E19E2B
:10396000700DF09E700D1124672F7727E61BF70B63
:10397000E29F8001E39F100DF29F100D1124E12FB3
:10398000722F4230510599F048F44115510569F004
:103990004130510581F0EB2F8D2F07C04430510588
:1039A00069F080F046305105B1F76E2F8DCFE22FD0
:1039B0007B2F812FFACFE22F7D2FF7CFEB2F822F96
:1039C000712FF3CF7B2F822FED2FEFCF41E00C949F
:1039D000511C08950C94E61CCF93DF93762FE901D8
:1039E000682F842F0E94EA1C798368838A83DF9181
:1039F000CF910895473908F046E90C94EC1C80916A
:103A00008D02982F9E7F61F48170826080938D0279
:103A100080919002873918F086E98093900208958A
:103A20008434B0F381708264F1CF88E090E00C942C
:103A3000F833CF92DF92EF92FF926B017C010E94EC
:103A4000FF1CB701A60188E090E0FF90EF90DF90A7
:103A5000CF900C94163460918D0270918E028091FB
:103A60008F02909190020C94191DEDE8F2E083E032
:103A7000808311828FEF828386E983831482608141
:103A80007181828193810C94191D8091440280FF81
:103A900076C08BE798E09F938F930E9443078091B5
:103AA00044020F900F9080FF6AC080918D02817058
:103AB0001F928F938EE598E09F938F930E94430708
:103AC000809144020F900F900F900F9080FF57C08D
:103AD00080918D0286951F928F9383E498E09F9347
:103AE0008F930E944307809144020F900F900F9094
:103AF0000F9080FF44C080918E021F928F9389E2C5
:103B000098E09F938F930E944307809144020F9007
:103B10000F900F900F9080FF32C080918F021F9204
:103B20008F938FE098E09F938F930E94430780913B
:103B300044020F900F900F900F9080FF20C0809153
:103B400090021F928F9385EF97E09F938F930E942F
:103B50004307809144020F900F900F900F9080FFC9
:103B60000EC0809191021F928F9389ED97E09F93F1
:103B70008F930E9443070F900F900F900F9008951E
:103B800080918D0280FF02C08695089580E008959F
:103B900090919102933018F49F5F90939102882343
:103BA00051F060918D0270918E0280918F02909100
:103BB00090020C94191D089581E00C94C81D9091F9
:103BC0009102992319F0915090939102882351F01A
:103BD00060918D0270918E0280918F02909190027F
:103BE0000C94191D089581E00C94DF1D80919102C1
:103BF0000895809391026623E9F060918D0270919F
:103C00008E0280918F02909190020E94191D8091E6
:103C1000440280FF0EC0809191021F928F9384E531
:103C200095E09F938F930E9443070F900F900F9002
:103C30000F9008959091440290FFFBCF1F928F93B5
:103C400081E395E0EECF60E00C94F91D80918E0247
:103C5000089580918F02089580919002089570E0F8
:103C60000C94232460911D0180918D0280FF0AC075
:103C700080911C0123E0829FC00111248E569D4F2C
:103C80000C942F1E80911E0190911F0123E0829FB2
:103C9000F0011124EE56FD4F891750F71182108262
:103CA00012828F5F3396F8CF90918D0290FF14C0EF
:103CB00090911E0120911F0133E0939FF001112488
:103CC000EE56FD4F921710F00C94321E81836083E4
:103CD00042839F5F3396F6CF0895CF93DF9300D052
:103CE0000F92CDB7DEB790918D0290FF0AC09E0172
:103CF0002F5F3F4F0E94FA1C4B8169818A810E948D
:103D0000541E0F900F900F90DF91CF910895CF9395
:103D1000DF93EC01EC81F0E0EC55F74F4491EDE8D6
:103D2000F2E0628181810E946D1E8C818F5F8C83A5
:103D3000DF91CF910895CF93DF93EC01EDE8F2E0AE
:103D4000438162818C810E946D1E8C818F5F8C8388
:103D5000DF91CF9108954F925F926F927F928F92F1
:103D60009F92AF92BF92CF92DF92EF92FF920F930A
:103D70001F93CF93DF9300D00F92CDB7DEB7182FEC
:103D8000D62E042F722E90918D0290FF46C0E92FFF
:103D9000E695AE2FB0E0A756BE4F8C9180935E02A1
:103DA0009E7F923009F04DC09E012F5F3F4F812FC3
:103DB0000E94FA1C4B8169818A810E94541E1093D3
:103DC0008E02D0928F0200939002772009F49CC05B
:103DD00060918D0270918E0280918F02909190027D
:103DE0000E94191D8091440280FF17C080919002AB
:103DF0001F928F9380918F021F928F9380918E02DA
:103E00001F928F938CE995E09F938F930E944307B5
:103E10000FB6F894DEBF0FBECDBF0F900F900F907E
:103E2000DF91CF911F910F91FF90EF90DF90CF9096
:103E3000BF90AF909F908F907F906F905F904F90CA
:103E40000895823019F400919002B9CF863019F4A8
:103E500010918E02B4CF8930D9F3883109F0AFCFF9
:103E6000E8518E2F8170682E8E2F80958170C82E1C
:103E7000E695F0E0EC55F64FE590F490412CFF24E8
:103E800091ECA92E95E0B92E60912001461618F00C
:103E90000E94321E94CF842C912C8E9CC0018F9C4A
:103EA000900D9E9C900D112470E00E94AE33512E17
:103EB000611028C0560E8091440280FF11C0FF920D
:103EC000EF921F92CF921F925F921F924F92BF92DA
:103ED000AF920E9443070FB6F894DEBF0FBECDBF6E
:103EE00020911E01820E911C9401220F331F280D78
:103EF000391D2E563D4F402F6D2D852D0E94FA1CE9
:103F00004394C2CF561AD7CF8091440280FF85CF09
:103F10001F920F931F92DF921F921F9385E795E0E8
:103F200073CFEDE8F2E09181282F4381628188E030
:103F3000890F0C94AB1E81E00C94911FEDE8F2E028
:103F40009181282F4381628188EF890F0C94AB1EE9
:103F500081E00C949E1FEDE8F2E0628128E0620FA0
:103F600008F46FEF282F438181810C94AB1E81E010
:103F70000C94AB1FEDE8F2E0628128E0621B08F4CC
:103F800060E0282F438181810C94AB1E81E00C946A
:103F9000BA1FEDE8F2E0438128E0420F08F44FEF4A
:103FA000282F628181810C94AB1E81E00C94C91F83
:103FB000EDE8F2E0438128E0421B08F440E0282FBE
:103FC000628181810C94AB1E81E00C94D81F20E0AB
:103FD0000C94AB1EEF92FF921F93CF93DF93EC01F3
:103FE00010E0EE24EA94F12C60912001161770F095
:103FF0000E94321E9A818C8190FF27C08F5F8C8334
:10400000DF91CF911F91FF90EF90089520911E01B5
:10401000422F410F5527551FCA019A01220F331F06
:10402000280F391F2E563D4F70E0C7010E94C23342
:10403000962F8C814091900260918F02199F800D84
:1040400011240E94FA1C1F5FCFCF8150D8CFAF92AE
:10405000BF92CF92DF92EF92FF920F931F93CF9375
:10406000DF93FC0182810FEF80FF01E010E040E36D
:10407000A42E809120011817C8F00E94321E809152
:104080005602013009F055C0811102C08091200113
:10409000815080935602DF91CF911F910F91FF9035
:1040A000EF90DF90CF90BF90AF900895C0911E0128
:1040B000C12ED12CCC0DDD2DD11DCE01880F991F25
:1040C000C80FD91FCE56DD4F198218821A8234E0EC
:1040D000E32EF12CB12C809156028B0D81331CF113
:1040E0006A2D0E94A033892F082E000C990BC81648
:1040F000D90691F4809190028E9DA0018F9D500D64
:10410000112455954795559547959E0160918F02CD
:1041100080918E020E94FA1CB00EF1E0EF1AF108B5
:10412000D1F61F5FA6CF87FFDFCF90912001890FC7
:10413000DBCF90E001966091200170E00E94C233D5
:10414000A8CF0F931F93CF93DF9380911E0190917F
:104150001F0123E0829FF0011124EE56FD4F8917C5
:1041600040F1C0E0D3E060912001C61740F10E9409
:10417000321E20911A0180915502820F80935502C0
:1041800090911B01920F90931B01191654F4082E65
:10419000000C990B409120014150550B8417950755
:1041A0001CF0219520931A01DF91CF911F910F915F
:1041B00008951182108212828F5F3396D0CF0C2F18
:1041C00010E070E0C8010E94C23320911E01820FEE
:1041D000482F50E020915502022E000C330B02179D
:1041E0001307BCF020911B01022E000C330B20178B
:1041F00031077CF08D9F900111242E563D4F409148
:10420000900260918F0280918E020E94FA1CCF5F13
:10421000AACFFA01EE0FFF1FE40FF51FEE56FD4F78
:10422000118210821282F3CF60918D02669570E048
:104230004BE050E081E291E00E94E333892B19F4D6
:1042400081E080935F020E94042B90935802809338
:1042500057028091440280FF08C088E195E09F9357
:104260008F930E9443070F900F90089510925F0262
:104270008091440280FF08C08FEF94E09F938F935A
:104280000E9443070F900F90089590918D0290FF28
:1042900054C0917081113BC0926090938D0266234F
:1042A000E9F160918D0270918E0280918F02909160
:1042B00090020E94191D8091440280FF0FC08091DE
:1042C0008D0286951F928F938FE197E09F938F9336
:1042D0000E9443070F900F900F900F9060918D02F6
:1042E000669570E04BE050E081E291E00E94E3339C
:1042F000892B01F10E94362181E080935A0240917E
:10430000900260918F0280918E020C94E71F82329E
:1043100010F09264C2CF880F982BBFCF80914402D7
:1043200080FFDCCF80918D0286951F928F9381E074
:1043300097E0CCCF0E941421DFCF0895682F909191
:104340008D02969581E0890F823208F081E00C940D
:10435000452181E00C949E21682F90918D029695C5
:104360008FEF890F09F481E20C94452181E00C94D0
:10437000AC2161E00C94452180918D028160809395
:104380008D028091440280FF0DC01F9281E08F93C7
:1043900083E996E09F938F930E9443070F900F90BD
:1043A0000F900F9080918D0286950C94B92160E05A
:1043B0000C94452180915D02811160C0809144027E
:1043C00080FF14C082EC97E09F938F930E94430775
:1043D000809144020F900F9080FF08C08CEA97E014
:1043E0009F938F930E9443070F900F900E94A614F3
:1043F000811110C08091440280FF08C084E897E0DA
:104400009F938F930E9443070F900F900E944A152D
:104410000E94351D0E94151D60938D0270938E02BF
:1044200080938F02909390026E7FC1F4809144023A
:1044300080FF08C08BE397E09F938F930E94430710
:104440000F900F900E94351D0E94151D60938D02E4
:1044500070938E0280938F02909390020E94FF1CB3
:104460000E94451D10925F0280918D0280FF03C063
:1044700086950E94D72181E080935D020895809106
:104480008D02816080938D028091440280FF0DC077
:104490001F9281E08F938AE596E09F938F930E940D
:1044A00043070F900F900F900F9080918D0286958B
:1044B0000C94D72180918D028E7F80938D02609124
:1044C0008D0270918E0280918F02909190020E94D5
:1044D000191D8091440280FF0FC080918D02817070
:1044E0001F928F9382E296E09F938F930E944307DF
:1044F0000F900F900F900F900E9436212FEF80E7C2
:1045000092E0215080409040E1F700C000000C9400
:10451000321E8091440280FF10C080918D028095F0
:1045200081701F928F938AEC96E09F938F930E94E5
:1045300043070F900F900F900F9080918D0280FD98
:104540000C945A220C94BC2180918D028E7F809312
:104550008D028091440280FF0CC01F921F9288EE52
:1045600095E09F938F930E9443070F900F900F90B9
:104570000F900E9436212FEF80E792E0215080407B
:104580009040E1F700C000000C94321E0F931F937F
:10459000CF93DF9380915F02882309F46FC08091ED
:1045A0005E02E0918D02E695E81BE09359028230AD
:1045B00091F5F0E0E056F74FE491CE2FD0E007E818
:1045C0001EE180915A02882361F010925A020E94E3
:1045D000042B909358028093570210925C02109221
:1045E0005B020E94042BE0915702F09158028E1B4F
:1045F0009F0B8F3F9F4708F041C0EC0FFD1FF093CA
:104600005802E093570287E592E0F801DF91CF91DD
:104610001F910F910994863049F4F0E0E356F74F6B
:10462000E491CE2FD0E00BE91EE1CBCF893051F4DD
:10463000E695F0E0E656F74FE491CE2FD0E00AEE93
:104640001FE1BFCF8F3051F4E695F0E0E956F74F08
:10465000E491CE2FD0E007E210E2B3CFC0EDD7E077
:1046600009EE1CE1853109F0ACCFF0E0EC56F74FD4
:10467000E491CE2FD0E001EA10E2A3CFDF91CF91F9
:104680001F910F910895FA01811101C0FB01099456
:10469000CF93DF93C82FD62F0E94C01D8C1740F0F8
:1046A0000E94C01D8D1720F4DF91CF910C94A92199
:1046B0008C2FDF91CF910C94B9211F93CF93DF936F
:1046C000EC01FB011281112309F4BBC00E94F0131D
:1046D0008272CC3CFCE5DF0709F499C008F044C0C5
:1046E000C63CECE5DE0709F47EC0F0F4C33C9CE573
:1046F000D90709F46EC048F4C23CDC4509F466C031
:10470000812FDF91CF911F910895C43C9CE5D9077B
:1047100009F464C048EA5FE16BE97FE1C53CDC4530
:1047200079F70E94432348C0C93CFCE5DF0709F440
:1047300064C068F4C73CECE5DE0709F459C047EBF8
:104740005FE166EC7FE1C83CDC4559F3D9CFCA3C58
:104750009CE5D90709F456C043EF5DE16CED7DE1BE
:10476000CB3CDC45F1F2CCCFC13DFCE5DF0709F4E1
:104770005FC098F4CE3C9CE5D90709F451C008F419
:104780004BC0CF3CFCE5DF0709F44FC0C03DDC4522
:1047900009F0B6CF6EE089E045C0C43D9CE5D9077D
:1047A00009F44CC058F4C23DFCE5DF0709F443C0EE
:1047B000C33DDC4509F0A4CF10E0A2CFC53D9CE588
:1047C000D907D1F3CD35DD45B9F39ACF0E948922BF
:1047D000F3CF46EB51E269EA71E2A3CF49EA51E235
:1047E00066EB71E29ECF4BE95FE168EA7FE199CF2A
:1047F00046EC5FE167EB7FE194CF44EE5FE165ED6E
:104800007FE18FCF45ED5FE164EE7FE18ACF4CED34
:104810005DE163EF7DE185CF81E00E94B921CCCFDE
:1048200065E082E00E944823C7CF68E086E0FACFC7
:1048300064E18FE0F7CF67E185E1F4CF61E288E1E1
:10484000F1CF11E05DCF539A4BB1477F5BB1586018
:10485000EFB7F8949B01220F331F260F371F280F45
:10486000391F2817390741F4EFBF8FE594E001970E
:10487000F1F700C000000895DC016D91CD0178E0F2
:104880005BB9000000C067FF4BB9660F000000C0B5
:1048900000C000C04BB900C07A9591F7E2CF83E227
:1048A00090E00E94F033813289F484E290E00E942B
:1048B000F033803159F485E290E00E94F03391E0CA
:1048C000833209F090E0892F8170089580E0FCCF59
:1048D000CF93C82F6FEF811161E283E290E00E94D5
:1048E00004346FEFC11160E184E290E00E9404346F
:1048F0006FEFC11163E285E290E0CF910C94043434
:10490000089586E290E00E94F033682F70E090E016
:1049100080E0089586E290E00C94043480E00E94E8
:10492000682460E070E0CB010E948A240E9438264F
:104930000E94242781E00C9468240E9480240E9415
:104940004F24811102C00C948E240895CF93FB0153
:10495000C281CC2309F19C0122513F452031310510
:1049600020F582510E943427C0E08C2FCF9108950A
:1049700081E00E94F90F43E062E081E00E94520A68
:10498000F3CF81E00E94041043E062E081E00E94E6
:10499000520AEBCF82E0F6CF8031FFE59F0789F323
:1049A00081319F45B9F3C1E0E0CF8031EFE59E074B
:1049B000F9F281319F45C9F682E0DBCF2FEFFC0190
:1049C00020830895CF93DF93EC0188818138A9F08B
:1049D00028F4803871F0DF91CF910895823881F00A
:1049E0008338C9F70E94261E89830E94291E8A8364
:1049F000F2CF0E942C1E8983EECF0E94C01DFBCFF8
:104A00000E94F61DF8CFCF93DF93EC0188818138A7
:104A1000E1F028F4803869F0DF91CF910895823871
:104A200011F18338C9F70E942C1E482F6A818981B1
:104A300008C0D9810E94291EC82F0E94261E4D2F12
:104A40006C2FDF91CF910C94E71F89810E94D721B1
:104A50008981811104C0DF91CF910C94A422DF9150
:104A6000CF910C943F228981DF91CF910C94231E2A
:104A7000EF92FF920F931F93CF93DF93EC01062FDA
:104A8000DC01ED91CD01E150E33108F0ADC0F0E083
:104A9000EC5AFB4C0C94D633198289E08A83602F40
:104AA000CE01DF91CF911F910F91FF90EF900C9469
:104AB000FB2B8981823069F0833071F08130D9F429
:104AC0000E94102B0E94DC336A837B838C839D833E
:104AD000E6CF0E948124F6CF7E0110E0812F0E9454
:104AE0007A18F701928383831F5FF2E0EF0EF11CC7
:104AF0001430A1F7D4CF602FCE010E94DE24CFCF97
:104B000089818230C1F76A817B818C819D810E947D
:104B1000DC330E948A24C3CF4B816A8189810E9441
:104B20000A269827892798279D838C83B8CF2C81C4
:104B30003D813227232732274B816A8189810E9458
:104B40002326ADCF0E943826AACF0E940325A7CFE7
:104B50000E94E224A4CF0E942B1DA1CF0E94CD264B
:104B600089839DCF0E94CF269827892798279A83EB
:104B7000898395CF6B8170E089819A81AE014C5F0A
:104B80005F4F9827892798270E94D22688CF6B816C
:104B900070E089819A81AE014C5F5F4F9827892729
:104BA00098270E94F9267BCF0E94242778CF0E9465
:104BB000F725D6CF6B8170E089819A81AE014C5F79
:104BC0005F4F9827892798270E94702668CF6B81AE
:104BD00070E089819A81AE014C5F5F4F98278927E9
:104BE00098270E9496265BCF8FEF888358CF84E06A
:104BF000089520E2629FB001112450E0440F551F38
:104C0000640F751F20E8829FC0011124860F971F33
:104C1000879608950F931F93CF93DF930E94F925F2
:104C20008C010E94F033C82FD0E0DC2FCC27C801C4
:104C300001960E94F0339E01282BC901DF91CF918C
:104C40001F910F9108950F931F93CF93DF93122F0E
:104C5000032F0E94F925EC01602F0E940434612F7C
:104C6000CE010196DF91CF911F910F910C940434E6
:104C7000AF92BF92CF92DF92EF92FF921F93CF93AA
:104C8000DF938CE8C82E81E0D82ED0E07601C0E01A
:104C900014C0F50125913491412F6C2F8D2F0E9466
:104CA000232682E0A80EB11C1F5F103191F780E22D
:104CB000E80EF11CCF5FC43019F0570110E0E9CFC6
:104CC000DF5F80E8C80ED11CD43001F7DF91CF91AF
:104CD0001F91FF90EF90DF90CF90BF90AF9008951D
:104CE000EF92FF920F931F93CF93DF93EC018A0112
:104CF0007C01E60EF71ECE018796CE15DF0539F44E
:104D0000DF91CF911F910F91FF90EF900895C11502
:104D100022E0D20740F40E94F033F80180830F5F55
:104D20001F4F2196E8CFF8011082F9CFCF92DF9282
:104D3000EF92FF920F931F93CF93DF937C016A0151
:104D40008C01060F171FEC01CE018796C017D10703
:104D500049F4DF91CF911F910F91FF90EF90DF9079
:104D6000CF900895C11522E0D20740F4FE01EE195C
:104D7000FF09EC0DFD1D60810E9404342196E4CFF3
:104D8000462F843038F4743028F4603118F4672FDB
:104D90000C940A2690E080E0089580E1089589ED62
:104DA00091E00895EF92FF920F931F93CF93DF93BB
:104DB000EC018A017C01E60EF71ECE01895D9D4F54
:104DC000CE15DF0539F4DF91CF911F910F91FF9040
:104DD000EF900895C93D21E0D20740F40E94F033DE
:104DE000F80180830F5F1F4F2196E7CFF8011082F3
:104DF000F9CFCF92DF92EF92FF920F931F93CF9351
:104E0000DF937C016A018C01060F171FEC01CE01B4
:104E1000895D9D4FC017D10749F4DF91CF911F9154
:104E20000F91FF90EF90DF90CF900895C93D21E062
:104E3000D20740F4FE01EE19FF09EC0DFD1D608163
:104E40000E9404342196E3CFCF93DF93C7E2D2E0F0
:104E500060E0CE010E9404342196C11584E0D80799
:104E6000B9F7DF91CF910895DF92EF92FF920F9300
:104E70001F93CF93DF9300D000D0CDB7DEB7F82ECD
:104E80008FE08F1540F08FEF93E00E94F03307E240
:104E900012E08823C1F00F900F900F900F90DF91D8
:104EA000CF911F910F91FF90EF90DF900895011522
:104EB00084E0180781F3C8010E94F033811101C01A
:104EC000FA940F5F1F4FF110F2CF19821A821B82E2
:104ED0001C82DD24D39478018FEFE81AF80AC80108
:104EE0000E94F03389831A828823A9F29FEF980FDA
:104EF000933078F48A83D9820E5F1F4FC7010E94D6
:104F0000F0338B83882339F2CE0101960E94B70BD0
:104F1000E2CF8701F9CF0F931F93CF93DF93C42F75
:104F2000D22FFC0182818823C9F0409362020E9443
:104F3000042B909361028093600280E28C0F883092
:104F400008F050C0C77081E001C0880FCA95EAF729
:104F5000DF91CF911F910F910C94390D1091620246
:104F6000141335C080916002909161020E941C2B45
:104F70008A3F910560F5C0E2CD0F1D17B9F080E2C0
:104F8000810F883040F4177081E001C0880F1A95B6
:104F9000EAF70E94400DC83048F481E09D2F9770D9
:104FA00001C0880F9A95EAF70E94390D802F0E9460
:104FB000310DC830B8F4D77081E001C0880FDA95A0
:104FC000EAF7DF91CF911F910F910C94400D80E291
:104FD0008C0F883038F4C77081E001C0880FCA9503
:104FE000EAF7EFCFDF91CF911F910F9108950F93C3
:104FF0009C01CB01233F4CE5340759F1A8F4283D2F
:10500000FCE53F0701F1293D4CE53407D1F1273D8F
:105010003C4591F406E221EE41EE67ED7CE50E940D
:105020008B2780E00F910895253FFCE53F07E9F0CD
:10503000B0F0263F3C45F9F0FC018281882339F12C
:1050400010926202EFCF07E225EE45EE68ED7CE5B7
:10505000E6CF06E221EE40EE63EF7CE5E0CF07E22B
:1050600025EE44EE64EF7CE5DACF06E221EE42EE77
:1050700065EF7CE5D4CF07E225EE46EE66EF7CE5F2
:10508000CECF08E221E045EE69ED7CE5C8CF81E0B6
:10509000C9CFCF93DF93EC01FB018281882309F410
:1050A00019C1C230FCE5DF07C0F1C6319CE5D90764
:1050B00030F09E012A5F3C452930310570F50E9491
:1050C000B91490937C0280937B02C031ECE5DE073B
:1050D00009F4CFC008F05BC0C8308CE5D80709F4EC
:1050E000B6C088F5C430ECE5DE0709F4A8C0C0F40A
:1050F000C2308CE5D80709F49CC080917B028260A5
:10510000C330DC4509F498C080917B0290917C0209
:105110000E94C7140E94800F80E0DF91CF91089514
:1051200080917B028061C630ECE5DE0709F484C023
:1051300080917B028860C730DC4508F47DC0809197
:105140007B02806279C0CC308CE5D80709F489C035
:1051500070F480917B028C60CA30ECE5DE0709F4C4
:105160006BC008F478C080917B028E7F65C0CE3022
:105170008CE5D80709F479C080917B028B7FCF3012
:10518000DC4508F459C080917B028F7E55C0CB3F2F
:10519000ECE5DE0709F457C030F5C3318CE5D807DC
:1051A00009F46FC078F4C131ECE5DE0709F465C09D
:1051B000C231DC4509F0A8CF0E94800F80917B02AC
:1051C0008F773AC0C5318CE5D80709F462C008F47E
:1051D00076C080917C028160CA3FDC4509F094CFA3
:1051E00080937C0291CFCF3FFCE5DF0709F44DC0EF
:1051F00088F480917C028D7FCD3F9CE5D90781F3B7
:1052000080917C028E7FCE3FDC4550F380917C0202
:105210008360E6CFC130FDE5DF0709F459C008F42B
:1052200044C080E0C230DD4509F06ECF0E944C15CD
:105230006BCF80917B02816080937B0265CF8091F0
:105240007B028460F9CF80917C028260C9CF80911B
:105250007B028064F1CF0E94800F80917B02806886
:10526000EBCF80917B028D7FE7CF80917B02877FA0
:10527000E3CF80917B028F7DDFCF80917B028F7B9C
:10528000DBCF80917B02837FD7CF80917C028C7FA4
:10529000A7CF80917B0282FB992790F921E092278A
:1052A00090FB82F990FB83F9C7CF80917C02982F05
:1052B000909591708E7F892B90FB81F991CF0E9400
:1052C000800F90917B02892F97FB87F98058B4CF8C
:1052D00081E0ACCF81E021CFCF93DF93EB0186312A
:1052E0009C4511F50E94F0139A81992399F08A7ACE
:1052F00091E009F490E090936302811109C089E282
:105300000E9497130E94331480E0DF91CF9108959B
:1053100085E3F6CF80916302811104C089E20E9487
:105320009E13F0CF85E3FBCF81E0EFCF909369022E
:10533000809368020895E0916802F09169023097C5
:1053400021F00190F081E02D099480E00895EF9222
:10535000FF920F931F93CF93DF938C01E09168022C
:10536000F09169023097C1F10280F381E02D099537
:105370008091440282FF30C080FF04C081EB9AE03C
:105380000E94AA06D0E0C0E08BEAE82E8AE0F82E60
:105390008091440280FF0EC0F801EC0FFD1F808158
:1053A0001F928F93FF92EF920E9443070F900F90EE
:1053B0000F900F902196C830D10551F7809144028B
:1053C00080FF0AC089EA9AE0DF91CF911F910F9187
:1053D000FF90EF900C94AA06DF91CF911F910F914F
:1053E000FF90EF900895E0916802F0916902309784
:1053F00039F022E0DC012C930480F581E02D099442
:10540000089520916602309167022817390771F0DC
:105410009093670280936602E0916802F0916902BE
:10542000309721F00680F781E02D099408952091AE
:105430006402309165022817390771F09093650274
:1054400080936402E0916802F0916902309721F044
:105450000084F185E02D099408959C012E5F3F4F53
:10546000AC01485F5F4F80E02417350709F40895C9
:10547000F90191919F019923B9F38F5FF5CF6623CD
:1054800049F0FC01329608962191261729F0E81779
:10549000F907D1F780E0089581E008959C01FC01AF
:1054A00032969FEF80E04191461751F09F3F19F4EB
:1054B000411101C0982F8F5F8630A9F79F3F09F4F3
:1054C0000895290F311D97FD3A95F90162830895DA
:1054D000FC01329608962191261303C0DF01119733
:1054E0001C92E817F907B9F708950C944E2A0C940A
:1054F000682A029626E0FC0111922A95E9F70895A0
:105500000895089508950C94822A80912A03843086
:1055100049F10E94832A80E00E94E70B10926A0200
:1055200088E190E020E40FB6F894A895809360009D
:105530000FBE2093600083B7817F846083BF83B7F1
:10554000816083BF7894889583B78E7F83BF0FB6C1
:10555000F894A89580916000886180936000109213
:1055600060000FBE08950895CF930E94812A0E9483
:10557000EC180E94B32AC0E08C2F0E947A18892B65
:1055800031F4CF5FC430C1F780E0CF91089581E05E
:10559000FCCF08950C94C92A0E94800F0E949B2979
:1055A0000E94E70B0C94CA2A1F921FB61F92112467
:1055B0008F939F93AF93BF9380916A02811113C021
:1055C0008091220390912303A0912403B09125039D
:1055D0004196A11DB11D8093220390932303A093B4
:1055E0002403B0932503BF91AF919F918F911F909A
:1055F0001FBE1F90189582E084BD93E095BD9AEF81
:1056000097BD80936E0008952FB7F8948091220380
:1056100090912303A0912403B09125032FBF0895F7
:105620002FB7F89460912203709123038091240393
:10563000909125032FBF08959C014FB7F894809156
:10564000220390912303A0912403B09125034FBF1F
:10565000821B930B089578941F921FB61F921124FA
:105660008F939F93AF93BF938091220390912303D5
:10567000A0912403B09125030196A11DB11D809333
:10568000220390932303A0932403B0932503BF9197
:10569000AF919F918F911F901FBE1F90189581E031
:1056A0008093E00080E28093D8001092C9008FE1DF
:1056B0009EE40197F1F700C0000087E090EBDC0169
:1056C0008093330390933403A0933503B093360350
:1056D00088E19CE00FB6F894A895809360000FBE17
:1056E00090936000FFCF9093D1018093D0010895F3
:1056F00080917902089590912A03943029F580933E
:105700006D0270936F0260936E029093E9008FEFC9
:105710009091E800815095FD06C095ED9A95F1F7BE
:1057200000008111F5CF8091E80085FF0DC050E0A9
:1057300040E063E070E08DE692E00E94B52E80913B
:10574000E8008E778093E8000895BC0184E00C9413
:105750007B2BBC0183E00C947B2B9C0184E0809329
:10576000E9009FEF8091E800915085FD06C085ED2E
:105770008A95F1F700009111F5CF8091E80085FF3F
:105780000CC050E040E066E070E0C9010E94B52E18
:105790008091E8008E778093E8000895CF93DF939F
:1057A000EC0181E08093E9008FEF9091E800815057
:1057B00095FD06C095ED9A95F1F700008111F5CFA2
:1057C0008091E80085FF14C050E040E068E070E0A0
:1057D000CE010E94B52E8091E8008E778093E8007C
:1057E00088E0FE01A1E7B2E001900D928A95E1F711
:1057F000DF91CF910895CF93FC01603221F5809124
:105800002A03843001F5C091E900CF702091EC00AB
:10581000922F917020FD90E8C92B82E08093E900DF
:105820008091E80080FF0CC050E040E060E270E052
:10583000CF010E94B52E8091E8008E778093E8001A
:10584000CF70C093E900CF91089588EE9AE00E944E
:10585000AA0680912903811109C00E9494300E94F8
:10586000F1308091E20084608093E200089584EE3C
:105870009AE00E94AA0610922903089580EE9AE009
:105880000C94AA068CED9AE00C94AA0688ED9AE096
:105890000C94AA0620916C022F5F822F62E30E9473
:1058A0009433992319F020936C02089510926C029E
:1058B000809170028823F1F080912A038430C1F432
:1058C0009091E9009F702091EC00822F817020FD63
:1058D00080E8892B95E09093E9009091EB0090FF90
:1058E00004C09091EE0097FD08C08F708093E9008E
:1058F0001092700208951092F1009091E80095FDC9
:10590000FACF9091E80090FFF0CF9091E8009E7759
:105910009093E800EACF42E061EC81E00E94103011
:1059200042E261EC84E00E94103042E261EC82E0ED
:105930000E94103042E260EC83E00E94103042E2AC
:1059400061EC85E00C94103080912C03833009F4D5
:1059500061C030F48130D1F1823009F49DC00895E6
:105960008A3009F489C08B3009F46FC0893009F09E
:1059700050C080912B03813209F04BC080912F03DE
:1059800090913003009719F0029709F042C080917E
:10599000E800877F8093E8008091E80082FF35C0AF
:1059A0009091F3008091F200029729F48091F10028
:1059B0008B7F813021F48091F10080937902809176
:1059C000E8008B778093E8000C94443080912B039F
:1059D000813AF9F48091E800877F8093E800809114
:1059E0002F0390913003892B61F468E081E792E006
:1059F00070E00E94532F8091E8008B778093E8003D
:105A0000089560E090E080E0F3CF80912A03811157
:105A1000C3CF089580912B03813AD9F780912F034A
:105A200090913003892BA9F78091E800877F8093BC
:105A3000E8008091E80080FFFCCF809136018093E0
:105A4000F1008091E8008E77BDCF80912B038132E9
:105A500001F780912F0390913003892BD1F680912B
:105A6000E800877F8093E8000E94443080912D03F6
:105A7000809336010C94800F80912B03813249F67C
:105A80008091E800877F8093E8000E9444308091F5
:105A90002E0380937A02089580912B03813A09F0B6
:105AA000B8CF8091E800877F8093E8008091E8007C
:105AB00080FFFCCF80917A02C2CF9FB7F8941092FA
:105AC00070029FBF90912A03943009F048C0209142
:105AD000E9002F703091EC00932F917030FD90E829
:105AE000922B25E02093E9002091EB0020FF34C0A9
:105AF0002091EE0027FF30C020916B02222321F07D
:105B00002091E80025FF28C010926B0226E030911A
:105B1000E80035FF14C08093F1008091E80085FD16
:105B200027C08091E80080FFFCCF8091E8008E774D
:105B30008093E8009F709093E90080E00895309191
:105B40002A03343049F43091EB0035FD05C0215073
:105B500041F481E080936B029F709093E9008FEF96
:105B60000895EFE9FFE03197F1F700C00000CFCFD3
:105B70008FB7F89421E0209370028FBFDBCF84B7FA
:105B8000877F84BF0FB6F894A895809160008861E4
:105B900080936000109260000FBE80E890E00FB626
:105BA000F89480936100909361000FBE0C9472157D
:105BB0000E9494300E94F130E2EEF0E08081846037
:105BC000808378940E9479330E9486158CE291E05C
:105BD0000E94962987EC9AE00C94AA06CF93DF9353
:105BE000CDB7DEB7A0970FB6F894DEBF0FBECDBF1E
:105BF00080912A03853051F483EC9AE00E94AA0632
:105C000080912A03853091F10E94CC2A0E94B81518
:105C100080912A03843009F583E08093E900809124
:105C2000E80082FF1AC08091E80090E085FF09C07B
:105C300050E040E060E270E0CE0101960E94042F47
:105C400091E08091E8008B778093E800992329F018
:105C500060E2CE0101960E943825A0960FB6F89416
:105C6000DEBF0FBECDBFDF91CF9108950E94852A80
:105C700080912803882321F20E94B42A882309F402
:105C8000BFCF0E949F2E0E94800FBACF0C94482E47
:105C9000292F33272330310521F168F421303105D4
:105CA00009F443C02230310509F444C090E080E09B
:105CB00030E020E026C02132310551F12232310599
:105CC000A9F76430710590F7FB01EE0FFF1FE15457
:105CD000FE4F2081318165547E4FFB01808190E031
:105CE00010C099278130910581F0009729F0029723
:105CF000E9F6ECEEFAE002C0EAE1FBE0849190E024
:105D00009F01FA01318320830895EAE0FBE0F6CF9A
:105D10006430710558F6660F771FFB01E953FE4F9B
:105D20002081318189E090E0ECCF82E190E029E9A7
:105D30003BE0E7CF8BE790E02EE13BE0E2CF80E174
:105D400089BD82E189BD09B400FEFDCF8091D800F4
:105D50008F7D8093D8008091E00082608093E00086
:105D60008091E00081FDFCCF0895AF92BF92CF9269
:105D7000DF92FF920F931F93CF93DF936C01EB01A0
:105D80008A010E946330F82E811123C0011511058C
:105D900039F0F80180819181C81BD90BC80ED91E3A
:105DA000B12CA12C2097A9F08091E80085FD22C09C
:105DB0008091E8008E778093E80001151105A1F02D
:105DC000F80180819181A80EB91EB182A08285E080
:105DD000F82E8F2DDF91CF911F910F91FF90DF90C3
:105DE000CF90BF90AF9008950E9463308823D1F286
:105DF000F82EEFCFF60181916F018093F10021978A
:105E0000FFEFAF1ABF0ACECFAF92BF92CF92DF9211
:105E1000FF920F931F93CF93DF936C01EB018A01E5
:105E20000E946330F82E811123C00115110539F04D
:105E3000F80180819181C81BD90BC80ED91EB12CE5
:105E4000A12C2097A9F08091E80085FD22C08091C7
:105E5000E8008B778093E80001151105A1F0F801A7
:105E600080819181A80EB91EB182A08285E0F82EB2
:105E70008F2DDF91CF911F910F91FF90DF90CF90E9
:105E8000BF90AF9008950E9463308823D1F2F82E1E
:105E9000EFCF8091F100F60181936F012197FFEF21
:105EA000AF1ABF0ACECFFC0180913103909132032B
:105EB00086179707A0F06115710529F49091E80005
:105EC0009E779093E80090E06115710551F491116F
:105ED00008C08091E80082FF34C080E00895BC01D2
:105EE000F2CF80912A038823C1F18530C1F18091DE
:105EF000E80083FD30C08091E80082FDEACF809108
:105F0000E80080FFE1CF8091F3002091F200382F6C
:105F10006115710519F02830310558F091E02830ED
:105F2000310509F090E02091E8002E772093E800F9
:105F3000CBCF81918093F100615071092F5F3F4F6A
:105F4000E7CF80912A03882341F0853041F080918A
:105F5000E80083FFBECF81E0089582E0089583E0EA
:105F60000895FC01809131039091320386179707C1
:105F7000A0F06115710529F48091E8008E77809377
:105F8000E80090E06115710551F4911108C080910D
:105F9000E80082FF35C080E00895BC01F2CF809117
:105FA0002A038823C9F18530C9F18091E80083FD77
:105FB00031C08091E80082FDEACF8091E80080FF47
:105FC000E1CF8091F3002091F200382F6115710527
:105FD00019F02830310558F091E02830310509F0EA
:105FE00090E08091E8008E778093E800CBCF849199
:105FF0008093F1003196615071092F5F3F4FE6CFDA
:1060000080912A03882341F0853041F08091E80097
:1060100083FFBDCF81E0089582E0089583E0089575
:10602000982F973028F08F708093E90081E00895D1
:106030009093E900242F762F50E0981731F070915B
:10604000EC002091ED005091F00021FD02C09F5F17
:10605000E8CF3091EB003E7F3093EB003091ED00C4
:106060003D7F3093ED003091EB0031603093EB00D9
:106070007093EC002093ED005093F0002091EE001F
:1060800027FDE5CF80E0089580912B0387FF13C0A3
:106090008091E80082FF06C08091E8008B778093B2
:1060A000E80004C080912A038111F2CF0895809105
:1060B0002A038823D9F38091E80080FFF8CF8091EC
:1060C000E8008E77ECCF2091E4003091E50095E672
:1060D000A9012091EC00822F817020FF06C08091E1
:1060E000E80080FF06C080E008952091E80022FDCE
:1060F0001AC080912A03882389F0853089F0809125
:10610000EB0085FD0FC02091E4003091E5004217BF
:106110005307F9F29150E1F684E0089582E0089582
:1061200083E0089581E008950E9402310E940A31BF
:10613000E0EEF0E0808181608083E8EDF0E0808136
:106140008F77808319BCA7EDB0E08C918E7F8C9304
:1061500080818F7E80831092290308950F931F936F
:10616000CF93DF930E9402310E940A31C8EDD0E044
:1061700088818F77888388818068888388818F7DF4
:10618000888319BC10922A031092260310922803C8
:106190001092270300EE10E0F80180818B7F80834E
:1061A00088818160888342E060E080E00E94103056
:1061B000E1EEF0E080818E7F8083E2EEF0E080818E
:1061C00081608083808188608083F80180818E7FF8
:1061D0008083888180618883DF91CF911F910F91A7
:1061E0000895E8EDF0E080818F7E8083E7EDF0E0B8
:1061F00080818160808384E082BF81E08093290375
:106200000C94AE30E8EDF0E080818E7F80831092B8
:10621000E20008951092DA001092E10008951F92B2
:106220000F920FB60F9211242F933F934F935F93CA
:106230006F937F938F939F93AF93BF93EF93FF934E
:106240008091E10082FF0BC08091E20082FF07C0D5
:106250008091E1008B7F8093E1000E944A2C809125
:10626000DA0080FF19C08091D80080FF15C08091AE
:10627000DA008E7F8093DA008091D90080FF96C08B
:1062800080E189BD82E189BD09B400FEFDCF81E0D6
:1062900080932A030E94252C8091E10080FF19C081
:1062A0008091E20080FF15C08091E2008E7F809394
:1062B000E2008091E20080618093E2008091D8004A
:1062C00080628093D80019BC85E080932A030E94E5
:1062D000422C8091E10084FF2BC08091E20084FF7A
:1062E00027C080E189BD82E189BD89B5982F917071
:1062F00080FFFBCF8091D8008F7D8093D800809164
:10630000E1008F7E8093E1008091E2008F7E809398
:10631000E2008091E20081608093E2008091260398
:10632000882309F449C084E080932A030E94462C04
:106330008091E10083FF29C08091E20083FF25C0A6
:106340008091E100877F8093E10082E080932A03BF
:10635000109226038091E1008E7F8093E10080916E
:10636000E2008E7F8093E2008091E2008061809362
:10637000E20042E060E080E00E9410308091F00096
:1063800088608093F0000E943E2CFF91EF91BF91B6
:10639000AF919F918F917F916F915F914F913F91BD
:1063A0002F910F900FBE0F901F90189519BC10924F
:1063B0002A030E94372C70CF8091E30087FD93E081
:1063C00090932A03B3CF1F920F920FB60F9211240E
:1063D0002F933F934F935F936F937F938F939F93ED
:1063E000AF93BF93CF93DF93EF93FF93D091E900E7
:1063F000DF708091EC00C82FC17080FDC0E8109262
:10640000E9008091F000877F8093F00078940E94EB
:1064100027321092E9008091F00088608093F000AC
:10642000CD2BCF70C093E900FF91EF91DF91CF9119
:10643000BF91AF919F918F917F916F915F914F919C
:106440003F912F910F900FBE0F901F9018951F93A3
:10645000CF93DF93CDB7DEB7AA970FB6F894DEBF20
:106460000FBECDBF8BE293E02091F100FC012193A0
:10647000CF01F3E083339F07B9F70E94A42C8091EA
:10648000E80083FF1EC180912B0390912C039A306A
:1064900008F017C1E92FF0E0E959FB4C0C94D63312
:1064A000803899F0823809F00CC180912F038F70E9
:1064B000873008F006C18093E9008091EB0085FBEE
:1064C000882780F91092E90006C0809127039091F7
:1064D0002803911182609091E800977F9093E800E3
:1064E0008093F1001092F1008091E8008E77E5C072
:1064F000882309F4D3C0823009F0E3C080912D03D2
:106500008111D6C080912F038F702FEF280F263076
:1065100008F0D7C08093E9002091EB0020FFC8C0AD
:10652000933031F48091EB0080628093EB00C0C027
:106530009091EB0090619093EB0021E030E001C07E
:10654000220F8A95EAF72093EA001092EA008091E0
:10655000EB008860EACF8111B4C010912D031F7742
:106560008091E3008078812B8093E3008091E800A4
:10657000877F8093E8000E9444308091E80080FF8C
:10658000FCCF8091E30080688093E30082E01111EA
:1065900083E080932A0395C08058823008F091C030
:1065A00080912D0390912E038C3D23E09207A1F55D
:1065B00083E08A838AE289834FB7F894DE011396D9
:1065C00020E03EE051E2E32FF0E050935700E491E9
:1065D00020FF03C0E295EF703F5FEF708E2F90E0D9
:1065E000EA30C0F0C7968D939D932F5F243159F701
:1065F0004FBF8091E800877F8093E8006AE270E0F7
:10660000CE0101960E94532F8091E8008B778093F2
:10661000E80057C0C096E7CF60912F037091300318
:10662000AE014F5F5F4F0E94462EBC01892B09F4DB
:1066300048C09091E800977F9093E80089819A8103
:106640000E94B12FE1CF8038E1F58091E800877F8B
:106650008093E800809126038093F10045CF81115B
:1066600030C090912D03923060F58091E800877FD3
:106670008093E800909326030E9444308091260383
:10668000882311F084E005C08091E30087FDFACFF4
:1066900081E080932A030E948B2C13C080912D03EC
:1066A000813079F481E0933009F080E08093280311
:1066B0001092E9008091E800877F8093E8000E94B3
:1066C00044308091E80083FF0AC08091E800877F12
:1066D0008093E8008091EB0080628093EB00AA96A3
:1066E0000FB6F894DEBF0FBECDBFDF91CF911F91E3
:1066F0000895CF9380912A038823A1F0C091E900E7
:10670000CF709091EC00892F817090FD80E8C82BAC
:106710001092E9008091E80083FD0E942732CF703B
:10672000C093E900CF910895991B79E004C0991FA7
:10673000961708F0961B881F7A95C9F780950895DB
:1067400087FB082E062687FD819567FD61950E94CF
:1067500094330EF4919507FC81950895AA1BBB1BF9
:1067600051E107C0AA1FBB1FA617B70710F0A61B51
:10677000B70B881F991F5A95A9F780959095BC0172
:10678000CD01089597FB072E16F4009407D077FDEE
:1067900009D00E94AE3307FC05D03EF49095819558
:1067A0009F4F0895709561957F4F0895EE0FFF1FDD
:1067B0000590F491E02D0994692796276927782799
:1067C000872778270895FC014150504030F0019010
:1067D0000616D1F73197CF01089588279927089594
:1067E000F999FECF92BD81BDF89A992780B5089599
:1067F000A6E1B0E044E050E00C942A34A8E1B0E017
:1068000042E050E00C942A34262FF999FECF92BD35
:1068100081BDF89A019700B4021639F01FBA20BD65
:106820000FB6F894FA9AF99A0FBE08950396272F97
:106830000E9405340E940434252F0E940534242F21
:106840000C9405340196272F0E9405340C940434CF
:10685000DC01CB01FC01F999FECF06C0F2BDE1BD20
:10686000F89A319600B40D9241505040B8F708950F
:10687000F894FFCF7E0D7E0DD60DD60D280E440E5A
:10688000AB0DAB0D4F0EB60EC50EC50E8F0F8F0F95
:10689000980F980F9A0F980F980F980F8F0F8F0FD0
:1068A0009F0F980F980F9F0F4C25592580258C25F9
:1068B0009725A225A525A825AB25F425F425AE25E9
:1068C000B225BA25C725D425D725DA25E7255032A4
:1068D0007832613378326133AB32CC326133233377
:0268E0002F3354
:1068E2002002FFFF2102FFFF2202FFFF2302FFFF20
:1068F20028022808641E140A321E010200300030E9
:10690200300118191A1B1C1D1E1F2021782BCE2B9B
:10691200AD2BA92BA52B01E200E900EA00B500B6D8
:1069220000B700CD008301CC008A019201940121BD
:1069320002230224022502260227022A02B300B4FD
:10694200006F007000818283E200E900EA00B50076
:10695200B600B700CD008301CC008A0192019401F8
:106962002102230224022502260227022A02B30060
:10697200B4006F00700081828300010202020206ED
:1069820006060909090909090F0F0F0F0F0F15153F
:10699200151818181818181818181840227B226A87
:1069A2000CCD0BEF0BAB0B300B490B690B820B00C1
:00000001FF
